:020000040000FA
:0C0000000000000016EF10F05DEF41F072
:0800180029EF42F0800E016E99
:10002000FE0EADD9010EABD9750E146E300E26EF53
:1000300002F0016A018E236EFE0EA1D923509FD1DA
:10004000076A800E3A6E00D01B6A1C6A1D6A1E6A1F
:10005000099AA0D9D8A01200D30FD8B4098A2D0FBD
:10006000C60FF7E20A0FF5E3176E166A156A146AEF
:100070000A0E136EBAEC02F0175013241B6E1450C4
:100080001C6E000ED8B0010E1C2615501D6E000E01
:10009000D8B0010E1D2616501E6E000ED8B0010EEF
:1000A0001E26070607E076D9D8A01200C60F02E286
:1000B0000A0FDAE209AA0BD01B1E1C1E1D1E1E1EF3
:1000C0001B2AD8B41C2AD8B41D2AD8B41E2A1B5007
:1000D000D880120030D803D0076A1B6E1C6A0096C5
:1000E0000750D8B40086050E066E270E186E100E47
:1000F0000CD8030E186EE80E08D8186A640E05D8DE
:10010000186A0A0E02D81B5007D0176E1C50146EC6
:100110001B50136EDDD91350136E064E0096075018
:1001200002E0065C07E21350D8A4009600B602D0A5
:10013000300F25D112001CAE12001B501C10D8B479
:1001400012001B1E1C1E1B4A1C2A2D0E18D13C6EB1
:1001500027AE02D02D0E13D9293E04D0283E02D05E
:10016000274A272A326A336A346A356A278E6A0E2A
:100170002626D8902732283229323532343233328B
:100180003232263EF6D72950265C2926265E285094
:10019000275C2826275E076A38D82E0EF0D83D6ADD
:1001A000D8903234296E3334286E3434276E353487
:1001B000266E3D36D89029362836273626363D36E7
:1001C000325029263350D8B0333C28263450D8B08A
:1001D000343C27263550D8B0353C2626D8B03D3E95
:1001E000D89029362836273626363D363D50300FF2
:1001F000C6D829C032F028C033F027C034F026C05A
:1002000035F03C2ECCD7D89012000096075003E171
:1002100000860A0E076E29C016F028C015F027C008
:1002200014F026C013F0066A1E6A1D6A1C6A0A0EC4
:100230001B6E23D9062A0650075CF6E11B50D8A492
:10024000009600A602D0072C03D01B50300F97D881
:10025000072EE1D712001B6E0650D8B412001BC047
:10026000E9FF1CC0EAFFEF50D8B4120088D81B4A3F
:100270001C2A0606F1D7A66AA68E0900F55002E0F0
:1002800002D8FBD71200206E8998899A9298929A88
:10029000F00E9216205000B21ED03A0E146E980E38
:1002A000D5D8330E1F6E29D8130E146E880ECED8F3
:1002B00024D8640ECAD821D8640EC7D8220E1F6E67
:1002C0001CD8280E07D80C0E05D8060E03D80082BD
:1002D000205001D000801F6E00A009D0899A030829
:1002E0000AE309D8090E146EC40EB0D812000080BB
:1002F000FE0818E0898A1F3A00A000908988F00E55
:1003000080161F500F0B8012000000D0000000006C
:1003100089981F3A000000D00000000000B0EDD71F
:10032000960E93D82050120002C013F008C014F0AB
:10033000176A186A000000D000009EBA11D0E86861
:100340001726182213221422D8A012001748183C8E
:10035000F1D7D00E176E030E186EEED79EAAFED7F9
:10036000AE50D8801200A66AA68E0900F55002E0B1
:1003700002D8FBD712009EA8FED7AD6E120001BEB8
:1003800082D701B4F8D701A205D001B003D001B2E1
:10039000EE6E12003AAE03D0EE50D88012003A5200
:1003A000C3E03A04DBE0A86EF2CFF3FFF29EA66A48
:1003B000A684550EA76EAA0EA76EA682A6B2FED779
:1003C000A694A94AAA2AF3BEF28EA68E1200A96E9E
:1003D000A66AA680A850A94AAA2AA68E1200080ECC
:1003E0001F6EEA6803C0E9FF045009B41CD909A4D0
:1003F0001CD9E26803C0E1FF0250120FE96E081C2D
:10040000EF161F500EE009B0F6D802C0E9FF143213
:100410001332EF500810D8A00818EF6E03D81F2E23
:10042000F6D712000450E71A000000D0E71A1200B5
:10043000186A176EFF0E1726182200D0D8A01200D7
:10044000030E146EE60E02D8F5D7146AFE0F136E73
:10045000000000D000D0E86A145AD8A01200130699
:1004600000D000D0F5D7010F206E0A0E176E186A63
:100470002FD8202EFDD71B5012002E6A2F6A306A0B
:10048000316A210E196E15D02E362F3630363136A0
:100490001B502E5C1C502F581D5030581E50315888
:1004A00008E3316E1B502E5E1C502F5A1D50305ADF
:1004B000D8801336143615361636192EE5D731C0C6
:1004C0001EF030C01DF02FC01CF02E501B6E12000D
:1004D0001C6A1B6A100EF36E14341B361C36175040
:1004E0001B5C18501C5805E317501B5E18501C5A13
:1004F000D88013361436F32EEFD713501200225043
:100500001C18800BF46E22AE05D0211E221E212A5B
:10051000D8B4222A1CAE05D01B1E1C1E1B2AD8B420
:100520001C2A176A136A146A186A1C5002E11B50CD
:1005300018E0100EF36ED890213622361736183692
:100540001C50185C02E11B50175C07E31B50175E40
:10055000D8A018061C50185ED88013361436F32E17
:10056000EAD7F4AE05D0131E141E132AD8B4142AE9
:100570001350120016C031F015C030F014C02FF027
:1005800013C02EF030501B02F3CF15F0F4CF16F04D
:100590002F501C02F3501526F45016222E501D0227
:1005A000F3501526F450162231501B02F350162634
:1005B00030501C02F35016262F501D02F350162601
:1005C0002E501E02F35016262E501B02F3CF13F0AE
:1005D000F4CF14F02F501B02F3501426F4501522C0
:1005E000000E16222E501C02F3501426F450152231
:1005F000000E16221200176A186A04D01432133241
:1006000017361836FF0FFAE218C014F01750136EA1
:100610001200136E14BE02D813501200131E141EC3
:10062000134A142A1200EF1203D0FF0AEF1601D06A
:10063000FF0AE988E92AEC161200FE0EDBCFE6FF7E
:10064000FF0EDBCFE6FFDD52DD521200A66AA68E5A
:100650000900F55002E0EE6EFBD71200E752E6CF3C
:10066000EEFF02E0E82EFAD71200F34E02D0E65277
:10067000FCD7E6CFEEFFE82EFCD71200E466FED7EB
:10068000F36EE552F32EFDD7E6CFEEFFE82EFCD752
:100690001200A66AA68EEE500900F55C02E1F5662E
:1006A000FAD71200A66AA68EEE500900F55C03E1A7
:1006B000F566FAD7010C000CA66AA68EEE5009006A
:1006C000F55C03E1F566FAD7000C010C316A35C020
:1006D00016F034C015F033C014F03250136E05E03C
:1006E00033AE03D03180800E141A14BE21D0010E17
:1006F000165C000E1558000E14587F0E135818E3A0
:10070000356A346A336A7F0E326E16C039F015C00E
:1007100038F014C037F013C036F009EC08F035C0DB
:1007200016F034C015F033C014F032C013F031822B
:100730000A0E356E890E346E340E336E7C0E326EB8
:1007400016C039F015C038F014C037F013C036F0B9
:100750006FEC08F016C039F015C038F014C037F04F
:1007600013C036F06FEC08F07C0E396E790E386EDF
:10077000350E376E810E366E7BEC07F016C039F001
:1007800015C038F014C037F013C036F06FEC08F025
:1007900016C039F015C038F014C037F013C036F069
:1007A0006FEC08F03F0E396E020E386E330E376E66
:1007B000830E366E7BEC07F016C039F015C038F0AA
:1007C00014C037F013C036F06FEC08F016C039F0E3
:1007D00015C038F014C037F013C036F06FEC08F0D5
:1007E000330E396E8C0E386E1E0E376E830E366EDB
:1007F0007BEC07F035C01AF034C019F033C018F0A4
:1008000032C017F01650356E1550346E1450336EDA
:100810001350326E16C039F015C038F014C037F0DE
:1008200013C036F06FEC08F01B0E396EE40E386E14
:10083000350E376E820E366E7BEC07F016C039F03F
:1008400015C038F014C037F013C036F06FEC08F064
:1008500016C039F015C038F014C037F013C036F0A8
:100860006FEC08F0A40E396EDB0E386E670E376E33
:10087000830E366E7BEC07F016C039F015C038F0E9
:1008800014C037F013C036F06FEC08F016C039F022
:1008900015C038F014C037F013C036F06FEC08F014
:1008A000330E396E8C0E386E1E0E376E830E366E1A
:1008B0007BEC07F035C01EF034C01DF033C01CF0D7
:1008C00032C01BF016C035F015C034F014C033F040
:1008D00013C032F01AC039F019C038F018C037F020
:1008E00017C036F06FEC08F01EC039F01DC038F0AC
:1008F0001CC037F01BC036F009EC08F035C039F0E9
:1009000034C038F033C037F032C036F031A20AD0EC
:10091000DB0E356E0F0E346E490E336E7F0E326E67
:1009200079EC07F031A002D0800E331A3550120056
:10093000010E1B6E3EC01DF03E8C1E6A1B6602D06F
:1009400033BE1E8E339E880E32603E8A35C013F051
:1009500034C014F033C015F032C016F0830E396E77
:10096000F90E386E220E376E7F0E366E6FEC08F081
:10097000BDEC08F032A004D0322A000E332234221B
:10098000070E32141C6E030E1C6404D0800E1E1A57
:10099000040E1C5E356A1CEC09F032501A6E6DE0D4
:1009A00035C017F034C018F033C019F0396A0F0E93
:1009B000386EC90E376E7E0E366E6FEC08F013C0BF
:1009C00039F014C038F015C037F016C036F07BECA3
:1009D00007F035C013F034C014F033C015F032C046
:1009E00016F017C035F018C034F019C033F01AC033
:1009F00032F0396AA20E386EDA0E376E6E0E366E2F
:100A00006FEC08F013C039F014C038F015C037F09F
:100A100016C036F07BEC07F035C013F034C014F08C
:100A200033C015F032C016F017C035F018C034F0DE
:100A300019C033F01AC032F0200E396EA20E386E93
:100A4000850E376E5C0E366E6FEC08F013C039F011
:100A500014C038F015C037F016C036F07BEC07F044
:100A60003250166E366E3350156E376E3450146E2B
:100A7000386E3550136E396E0CD01650326E366E9D
:100A80001550336E376E1450346E386E1350356E09
:100A9000396E6FEC08F035C017F034C018F033C071
:100AA00019F032C01AF01C301C18010B1B184EE054
:100AB000CE0E396EF50E386E4C0E376E6F0E366EEA
:100AC0006FEC08F01A0E396E060E386EB60E376EE1
:100AD000750E366E7BEC07F017C039F018C038F091
:100AE00019C037F01AC036F06FEC08F0A50E396E59
:100AF000AA0E386E2A0E376E7A0E366EFCD917C0E3
:100B000039F018C038F019C037F01AC036F06FEC61
:100B100008F017C039F018C038F019C037F01AC003
:100B200036F06FEC08F017C039F018C038F019C073
:100B300037F01AC036F036663606DBD93E9C396A85
:100B4000386A376A7F0E366ED6D956D0F90E396EAE
:100B5000680E386E360E376E6C0E366E6FEC08F01F
:100B6000C00E396E070E386ED00E376E720E366EAE
:100B7000C2D917C039F018C038F019C037F01AC000
:100B800036F06FEC08F0840E396E880E386E080E61
:100B9000376E780E366EAFD917C039F018C038F0FE
:100BA00019C037F01AC036F06FEC08F0AB0E396E92
:100BB000AA0E386E376E7C0E366E9DD917C039F08E
:100BC00018C038F019C037F01AC036F06FEC08F0D2
:100BD00013C039F014C038F015C037F016C036F025
:100BE0006FEC08F03E9C13C039F014C038F015C00B
:100BF00037F016C036F07FD9800E1B5202E01CB2CF
:100C00001E1A1EBE331A1DBC3E8C3550120033BE58
:100C1000A6D03252D8B4A4D032C01CF03EC01DF0D1
:100C20003E8C7F0E326E396A386A376A366E61D909
:100C300035C013F034C014F033C015F032C016F0D4
:100C4000130E396ECB0E386E030E376E840E366E71
:100C500052D913C039F014C038F015C037F016C09F
:100C600036F06FEC08F0BC0E396E5A0E386E050E79
:100C7000376E860E366E3FD913C039F014C038F087
:100C800015C037F016C036F06FEC08F0830E396EE1
:100C9000300E386E720E376E850E366E2CD935C01A
:100CA00017F034C018F033C019F032C01AF013C076
:100CB00035F014C034F015C033F016C032F08E0E8B
:100CC000396ED70E386E6B0E376E810E366E6FEC46
:100CD00008F0B50E396E290E386E4E0E376E840E42
:100CE000366E09D913C039F014C038F015C037F08A
:100CF00016C036F0F4D9800E396E300E386E720E92
:100D0000376E840E366EF7D817C039F018C038F039
:100D100019C037F01AC036F07CD913C039F014C0AE
:100D200038F015C037F016C036F0D9D9396A386AAC
:100D3000376A7F0E366EDFD81CB009D0F30E396EDD
:100D4000040E386E350E376E7F0E366EC8D97F0EA4
:100D50001C261C30326E1DBC03D03E9C01D03E8A46
:100D60003550120032503662000C33503762000C9E
:100D700034503862000C35503962000C010C375089
:100D80003318416E41BE30D037BE17D03650325C7A
:100D9000D8A0000CD8A4010C3750335CD8A0000CAC
:100DA000D8A4010C3850345CD8A0000CD8A4010C95
:100DB0003950355CD8A0000C010C3250365CD8A0FC
:100DC000000CD8A4010C3350375CD8A0000CD8A478
:100DD000010C3450385CD8A0000CD8A4010C35505C
:100DE000395CD8A0000C010C33AE010C000C37505C
:100DF0003318416E41BE34D037BE19D03650325C04
:100E0000D8A0000CD8A4010C3750335CD8A0000C3B
:100E1000D8A4010C3850345CD8A0000CD8A4010C24
:100E20003950355CD8A0000CD8A4010C000C32500D
:100E3000365CD8A0000CD8A4010C3350375CD8A085
:100E4000000CD8A4010C3450385CD8A0000CD8A4F5
:100E5000010C3550395CD8A0000CD8A4010C000C52
:100E600033AE010C000C33503718416E41BE34D004
:100E700033BE19D03250365CD8A0000CD8A4010C77
:100E80003350375CD8A0000CD8A4010C3450385C27
:100E9000D8A0000CD8A4010C3550395CD8A0000CA7
:100EA000D8A4010C000C3650325CD8A0000CD8A499
:100EB000010C3750335CD8A0000CD8A4010C38507A
:100EC000345CD8A0000CD8A4010C3950355CD8A0F3
:100ED000000CD8A4010C000C37AE010C000C396AD0
:100EE000386A7E0E366E800E33AE000E376E03D833
:100EF00044D1800E371A3650325C3D6E11E23D6CA3
:100F0000325036C032F0366E335037C033F0376E61
:100F1000345038C034F0386E355039C035F0396E41
:100F20001A0E3D6074D0365272E03C6A3350406E07
:100F300037183F6E338E378E080E3D5E08E339C09A
:100F40003CF038C039F037C038F0376AF5D73D2665
:100F500007E0D8903732383239323C323D2EF9D75B
:100F60003FAE33D03950355E3850345A3750335A4B
:100F700007E2D880000E355634563356800E401A9C
:100F80003C6C04E03506000E345A335A040E3D6EB4
:100F900033660DD034C033F035C034F03CC035F08A
:100FA0003C6A080E325E29E33D2EF2D726D033BECE
:100FB00008D0D8903C36353634363336322EF7D713
:100FC0001CD03CAE22D03C6A0FD039503526385068
:100FD00034223750332206E33332343235323C3256
:100FE000324A0DD03CAE11D0353E0FD0343E0DD03C
:100FF000333E0BD0D8803590EFD7326A02D03E8294
:101000003268356A346A800E336E40AE339E355096
:1010100012003350306E37183F6E365051E0325266
:1010200052E0325E7F0E03E2322603E24BD03226DC
:101030004CE235C02EF034C02FF0308E378E180EB3
:10104000406E356A346A336A0BD039502E5C3850A2
:101050002F5811E32F6E306A39502E5E0BD004E208
:101060003750305CF2E007E339502E5E38502F5A8B
:101070003750305AD8803536343633362E362F3600
:101080003036402EECD733BE07D032521BE03F3211
:101090003206402A3F36E3D707E239502E5E3850F9
:1010A0002F5A3750305A17E3353E15D0343E13D0FF
:1010B000333E11D0333234323532323E0CD005D08B
:1010C0003E8604D03E84326A02D03E823268356A5F
:1010D000346A800E336E3FAE339E3550120033506B
:1010E000306E37183F6E3250D8A436503AE0322670
:1010F0007E0E03E3325E03E336D0325E31E335C069
:101100002EF034C02FF0308E378E356A346A336A51
:10111000180E406E30322F322E3206E3395035260B
:101120003850342237503322333234323532402E65
:10113000F1D733BE07D0353634363336325210E06D
:101140003206303416E3353E14D0343E12D0333EEE
:1011500010D0D880333234323532323E0AD003D008
:101160003E84326A02D03E823268356A346A800E2A
:10117000336E3FAE339E3550120032C040F03350D4
:1011800035C033F0356E3536403235323E6A35364D
:10119000403602E33E843E7E06E13E80406A356A88
:1011A000346A336A0BD0402803E0D880353206D049
:1011B000D890353202E13E8201D03E863EB604D060
:1011C0003EA20FD03EB407D07F0E356EFF0E346EB8
:1011D000336E326E23D0800E356E01D0356A000E2C
:1011E000F6D73EB0FBD7326A9F0E4060EBD77E0E3B
:1011F0004064F4D79E0E405C07E0D890353234321C
:1012000033323232402AF6D73EA408D0D880000EBE
:10121000325633563456355635AEE0D7325012007A
:10122000000E33BEFF0E346E356E06D0326E336A5A
:10123000346A356A3F9E0AD03F9E35AE07D0D880CB
:10124000000E32563356345635563F8E960E406E4B
:10125000355209E0080E402633C032F034C033F076
:1012600035C034F011D034520FE1080E405E3350D7
:1012700007E1080E405E325002E1355010D0326A6C
:10128000346E32C033F0326A34BE06D0D890323673
:10129000333634364006F8D73FAE349E405032C025
:1012A00035F0326E345033C034F0336E12002020EB
:1012B000202050494331384634364B3232202020EA
:1012C0002020000020202020416E74656E6E612079
:1012D000526F746F72202020000020436F6E747272
:1012E0006F6C6C6572207665722E0000416E7465BD
:1012F0006E6E6120526F746F7220436F6E74726FE6
:101300006C6C657220762E20000056657273696FD2
:101310006E2000005061726B696E6720415A3D007B
:10132000417A696D757468206F66667365743D20D7
:101330000000417A696D757468206F666673657424
:101340002073617665640000456C65766174696F31
:101350006E206F66667365743D200000456C65768F
:101360006174696F6E206F66667365742073617651
:10137000656400002D2D2D2D2D2D2D2D2D2D2D2D88
:101380002D2D434F4D4D414E44204C4953542D2D4E
:101390002D2D2D2D2D2D2D2D2D2D2D2D00003F20D2
:1013A0002048656C7020546578740000412020430B
:1013B000572F43435720526F746174696F6E2053E7
:1013C000746F7000422020416E74656E6E6120441F
:1013D0006972656374696F6E20454C00432020413B
:1013E0006E74656E6E6120446972656374696F6EB8
:1013F00020415A00433220416E74656E6E61204474
:101400006972656374696F6E20415A26454C00000D
:10141000442020446F776E20446972656374696F5D
:101420006E20526F746174696F6E00004520205504
:10143000502F444F574E20446972656374696F6E34
:1014400020526F746174696F6E2053746F70000066
:10145000462020536574206D6178696D616C207041
:101460006F736974696F6E20696E20617A696D753A
:1014700074683A204661616100004621205361761C
:10148000652063757272656E7420706F736974691C
:101490006F6E206173206D6178696D616C20706F73
:1014A000736974696F6E0000463F2053686F772040
:1014B0006D6178696D616C20706F736974696F6EAE
:1014C00020696E20617A696D757468004720205329
:1014D0006574204F666673657420496E20454C3AEA
:1014E000204765656500473F2053686F77204F664A
:1014F0006673657420436F6E7374616E7420666FDB
:101500007220454C000048202048656C70207465AE
:101510007874000049202053686F772070617261F1
:101520006D657465727300004A44205365742042EF
:101530006565706572206F6E202D20446972656349
:10154000742043757272656E74004A462053657448
:1015500020426565706572206F6E202D2046726591
:101560007175656E637900004A4E205365742042A0
:101570006565706572206F6666004A6E20536574FB
:1015800020626565706572206672657175656E634F
:101590007920286E203D20313030302D31303030F0
:1015A0003020487A29004B2020416E74656E6E61B0
:1015B00020446972656374696F6E20536574746941
:1015C0006E6720496E20454C3A204B6565650000EA
:1015D0004C2020436F756E74657220436C6F636B93
:1015E0007769736520286C6566742920526F746171
:1015F00074696F6E00004D2020416E74656E6E61DF
:1016000020446972656374696F6E205365747469F0
:101610006E6720496E20415A3A204D616161000099
:101620004E202054797065206F6620646973706C59
:10163000617900004F20204F666673657420496E03
:1016400020415A004F3F2053686F77204F666673E2
:10165000657420436F6E7374616E74004F21205364
:101660006176652063757272656E7420706F736940
:1016700074696F6E2061732053544F5020706F73E4
:101680006974696F6E005020205061726B696E67DB
:1016900020546F3A205061616120656565005021DA
:1016A00020536176652063757272656E7420706F69
:1016B000736974696F6E206173207061726B696EFB
:1016C000672076616C7565730000503F2053686F2A
:1016D00077207361766564207061726B696E672034
:1016E00076616C75657300005120205072656369E6
:1016F00073696F6E20302E31202D20302E35202D35
:1017000020312E30206465670000522020436C6F2A
:10171000636B776973652028726967687429205242
:101720006F746174696F6E00532020416C6C20539C
:10173000746F7000546E20436F6D2E20706F727442
:1017400020737065656420286E3D343830302C3944
:101750003630302C31393230302C33383430302C74
:101760003537363030290000552020557020446927
:1017700072656374696F6E20526F746174696F6E05
:101780000000562020536F6674766172652056659E
:101790007273696F6E00572020416E74656E6E61C2
:1017A00020446972656374696F6E2053657474694F
:1017B0006E673A20576161612065656500005920B8
:1017C000204543484F204F4E202F204F46460000D3
:1017D0005A2020537769746368207A65726F20708D
:1017E0006F736974696F6E20746F204E6F7264201E
:1017F0002F20536F75746800262020536574206D68
:101800006178696D756D20656C65766174696F6E60
:101810002028313830202D20666C6970206F6E3B97
:10182000203930202D20666C6970206F6666290093
:10183000252020456C65766174696F6E20636F6E3C
:1018400074726F6C204F4E202F204F4646002A2086
:10185000204D61782E20656C65766174696F6E200D
:10186000666F72206F7665727475726E696E67004E
:10187000232020456D756C6174696F6E206F662042
:10188000475332333241202F204753323332420004
:101890003C2020417A696D7574682063616C6962CF
:1018A000726174696F6E00005E2020456C65766120
:1018B00074696F6E2063616C6962726174696F6EC6
:1018C00000005B20204F776E20636F6F7264696E3B
:1018D000617465202D206C61746974756465000005
:1018E0005D20204F776E20636F6F7264696E617444
:1018F00065202D206C6F6E67697475646500616189
:101900006120497320416E2056616C756520466FD9
:10191000722054686520417A696D7574682028309A
:101920002D333630290065656520497320416E20CE
:1019300056616C756520466F722054686520456C51
:1019400065766174696F6E2028302D31383029003A
:10195000446973706C617920747970652000302E51
:101960003500302E3100312E3000302E32005072D2
:1019700065636973696F6E2073657420746F2000EE
:101980005A65726F20706F736974696F6E206F6E25
:1019900020004D6178696D756D20656C65766174A8
:1019A000696F6E2069732000426565706572000082
:1019B0003A204672657175656E6379003A20446914
:1019C000726563742063757272656E7400002066C0
:1019D00072657175656E63793A200000434F4D2042
:1019E000706F72742073706565643A2000005468EB
:1019F000652073706565642077696C6C206F6E6C10
:101A0000792062652076616C696420616674657214
:101A1000207265626F6F7400434F4D20737065656F
:101A200064206973206E6F74207265636F6D6D65DD
:101A30006E6465642E20596F7520626574746572DA
:101A40002075736520343830302C393630302C31E5
:101A5000393230302C33383430302C353736303062
:101A600000005265626F6F74206E6F773F20287997
:101A7000203D20796573206F74686572203D206E6B
:101A80006F2900004E657720434F4D2073706565C8
:101A9000642061637469766174656400456C657681
:101AA0006174696F6E20697320004D6178696D758E
:101AB0006D206F6620617A696D7574683D20000045
:101AC00056616C7565207361766564005479706544
:101AD0003A204753323332002D2D2D2D2D2D2D4CF4
:101AE000495354204F4620504152414D4554455290
:101AF000532D2D2D2D2D2D2D00004F6666736574F1
:101B0000206F6620617A696D7574683A20004F66AF
:101B100066736574206F6620656C65766174696FA5
:101B20006E3A20004D6178696D756D20706F736934
:101B300074696F6E206F6620617A696D7574683A9A
:101B400020004D6178696D756D20706F73697469DF
:101B50006F6E206F6620656C65766174696F6E3A92
:101B600020004D61782E20656C65766174696F6E1A
:101B700020666F72206F7665727475726E696E671B
:101B80003A200000456C65766174696F6E20636F62
:101B90006E74726F6C3A20005061726B696E6720D0
:101BA0006F6E20415A3A20005A65726F20706F7331
:101BB0006974696F6E3A2000434F4D20706F7274E4
:101BC000206563686F3A20004265657065723A204F
:101BD00000004672657175656E63790044697265CF
:101BE00063742043757272656E740000426565709F
:101BF0006572206672657175656E63793A200000C2
:101C0000507265636973696F6E3A2000446973703E
:101C10006C617920747970653A2000004C617469B8
:101C2000747564653A20000020204C6F6E676974FB
:101C30007564653A2000536F66747761726520762B
:101C4000657273696F6E3A200000464552523A2021
:101C50000000204F4552523A200041726520796FB2
:101C60007520737572653F00417A696D75746820DF
:101C700069732063616C6962726174656400417AA2
:101C8000696D7574682063616C6962726174696EF4
:101C900067206572726F7200456C65766174696F5A
:101CA0006E2069732063616C69627261746564009F
:101CB000456C65766174696F6E2063616C696272F0
:101CC0006174696E67206572726F72006C6174690D
:101CD000747564653A2000006C6F6E676974756492
:101CE000653A2000454C3A204572726F7200415AA5
:101CF0003A204572726F7200444F574E2055502063
:101D000053544F5020434357202043570000415A1B
:101D1000494D5554483A2000415A494D5554483A86
:101D2000204572726F722020202020200000202089
:101D300020202020202053544F5020434357202060
:101D40004357000020202020202020204D454E55C4
:101D500020202020202020200000202020202020C3
:101D600020202020202020202020202020200000B3
:101D700053455420415A494D55544820544F202032
:101D8000000053455420454C455641542E20544F95
:101D9000202000005041524B494E4720415A494DA6
:101DA0005554482000005041524B2E20454C45567A
:101DB0004154494F4E200000415A494D5554482046
:101DC0004F464653455420200000454C455641544B
:101DD0002E204F4646534554202000004D4158497F
:101DE0004D554D20415A494D5554482000004D4114
:101DF0005820454C202D204F564552542E2000008F
:101E000054595045204F4620444953504C41592085
:101E1000200020204C454420204C43440000454CE9
:101E200045564154494F4E20434F4E54522E2000A8
:101E3000434F4D4D554E49434154494F4E20475312
:101E40003233320020202041202020204220000078
:101E50004D4158494D554D20454C455641542E2035
:101E600000002020203930202031383000005A4531
:101E7000524F20504F494E54204F4E2000004E4F9D
:101E8000524420200000534F555448200000202089
:101E900020204E202020532000004245455045522E
:101EA000202020004F4646202020202020202000F7
:101EB000446972656374204375722E004652455121
:101EC00055454E435920200020204F4646202044AF
:101ED00043202046525100004652455155454E433D
:101EE000593A202000002020202056657273696F27
:101EF0006E200000505245434953494F4E20200068
:101F0000302E3120646567202000302E3220646539
:101F100067202000302E3520646567202000312E98
:101F200030206465672020005345542041534C20E5
:101F3000544F202020004155544F205455524E49B3
:101F40004E472020202020004F5645525455524ED7
:101F5000494E4720202020202000434F4D20535041
:101F600045454420202020202000434F4D20504F45
:101F70005254204543484F20495320004E4D45417F
:101F8000205445535420202020202020200043416D
:101F90004C4942524154494F4E2020415A49204514
:101FA0004C450000202020415A4920454C45000066
:101FB00043414C4942524154494F4E20504C5320CA
:101FC00057414954000020202020202020200000DC
:101FD0002020202020202000474741002020204FA3
:101FE000464620204F4E00004C617469747564654C
:101FF0003A20202000004C6F6E6769747564653A62
:1020000020002020204F4B20202000003031323390
:10201000343536373839414243444546303132331E
:10202000343536373839414243444546400E3E6EDA
:10203000006AB886A00EAF6E010EB06E200EAC6EB8
:10204000900EAB6E000124EE47F00F01386B396B38
:102050003A6B3B6B3C6B796A786A606A03018E6B02
:102060008D6B100E8C6F830E8B6F0001896A8A6AEC
:102070008B6A8C6A8D6AC00E926E070E936EBE0ECE
:10208000946EF40E956E880E966E310ECD6EB16A1A
:10209000250E9D6EA06A0B0EBD6EFA0EBF6EBE6A57
:1020A000666AF40ED36E400E9B6EC00EF26E700E1A
:1020B000F16E900EF06E9F8A9F94D08EF188F0881A
:1020C000D26A080EB86E200EAC6E060EB06E820E8E
:1020D000AF6E900EAB6E716A726A796A786AC26A84
:1020E0000F0EC16EC06A0F01386B396B3A6B3B6BD8
:1020F0003C6B5D6B576BC66A6C6A02EE12F0120E97
:10210000F76EAE0EF66E26EC03F0EF6A0301010ED9
:10211000566F400E886F93988A9893968A96939AF2
:102120008A9A939C8A9C95968C9695928C9295907F
:102130008C9094908B90429E4390516B526B506B5D
:10214000449C429C439E336B326B316B306B376BDC
:10215000366B356B346B448283AC4492448483AEDB
:102160004494448844860001AA6BBD6BBC6BBF6B72
:10217000BE6B0301640E5B6F0001A76BA86B010EC1
:10218000966F810EDA6FED0EDB6F430EDC6F490E3A
:10219000DD6F2D0EDE6F190EDF6F110EE06FCD0EAD
:1021A000E16F010EE26F090EE36FE469170EE56F50
:1021B000930EE66F310EE76F750EE86F070EE96F4D
:1021C000130EEA6F850EEB6FF10EEC6F050EED6FDF
:1021D000B30EEE6F910EEF6F710EF06F770EF16F21
:1021E000330EF26FF70EF36F7F0EF46F610EF56F23
:1021F000640E18EC02F0FE0E43EC01F0400E43ECCE
:1022000001F0000E43EC01F0040E43EC01F0040E6B
:1022100043EC01F0040E43EC01F0150E43EC01F029
:102220000E0E43EC01F0040E43EC01F0000E43EC03
:1022300001F01E0E18EC02F0FE0E43EC01F0480E09
:1022400043EC01F0000E43EC01F0040E43EC01F00E
:102250000E0E43EC01F0150E43EC01F0040E43ECBE
:1022600001F0040E43EC01F0040E43EC01F0000E0B
:1022700043EC01F01E0E18EC02F0FE0E43EC01F0F0
:10228000500E43EC01F0000E43EC01F0040E43EC61
:1022900001F0020E43EC01F01F0E43EC01F0020EC0
:1022A00043EC01F0040E43EC01F0000E43EC01F0AE
:1022B000000E43EC01F01E0E18EC02F0FE0E43EC93
:1022C00001F0580E43EC01F0000E43EC01F0040E57
:1022D00043EC01F0080E43EC01F01F0E43EC01F05B
:1022E000080E43EC01F0040E43EC01F0000E43EC49
:1022F00001F0000E43EC01F01E0E18EC02F0FE0E91
:1023000043EC01F0600E43EC01F0000E43EC01F0F1
:10231000010E43EC01F0050E43EC01F0090E43EC15
:1023200001F01F0E43EC01F0080E43EC01F0040E27
:1023300043EC01F0000E43EC01F01E0E18EC02F02D
:10234000FE0E43EC01F0680E43EC01F0040E43EC8A
:1023500001F00A0E43EC01F0040E43EC01F0000E14
:1023600043EC01F0000E43EC01F0000E43EC01F0F1
:10237000000E43EC01F0000E43EC01F01E0E18ECD1
:1023800002F0AA6A210EA96EE8EC01F00301896F40
:10239000E8EC01F003018A6FAA6AA96AE8EC01F08F
:1023A0004A6EE8EC01F04B6EAA6A020EA96EE8ECE8
:1023B00001F04C6EE8EC01F04D6EAA6A040EA96EB5
:1023C000E8EC01F00001676FE8EC01F0686FAA6AC1
:1023D000060EA96EE8EC01F0696FE8EC01F06A6F97
:1023E000AA6A080EA96EE8EC01F06F6FE8EC01F044
:1023F000706FAA6A0A0EA96EE8EC01F0716FE8EC42
:1024000001F0726FAA6A0C0EA96EE8EC01F0736F0E
:10241000E8EC01F0746FAA6A0E0EA96EE8EC01F008
:10242000666FAA6A0F0EA96EE8EC01F09A6FAA6AAD
:102430001E0EA96EE8EC01F09B6FAA6A100EA96E41
:10244000E8EC01F00301596FAA6A110EA96EE8ECDD
:1024500001F00301556FAA6A1F0EA96EE8EC01F0A6
:102460000001B86FE8EC01F0B96FAA6A120EA96E0C
:10247000E8EC01F003013A6FE8EC01F003013B6F77
:10248000E8EC01F003013C6FE8EC01F003013D6F63
:10249000AA6A160EA96EE8EC01F003013E6FE8ECA3
:1024A00001F003013F6FE8EC01F00301406FE8EC3D
:1024B00001F00301416FAA6A1A0EA96EE8EC01F05F
:1024C0000301426FE8EC01F00301436FAA6A1C0E9E
:1024D000A96EE8EC01F00301856FE8EC01F003015F
:1024E000866F86510A0DF3CF86F385510A0DF3CF1F
:1024F00085F3F4508627166A070E156EA10E146E2A
:10250000200E136E85C31BF086C31CF01D6A1E6A65
:102510003DEC02F014C084F313C083F3020E0301F8
:10252000555DD8A4010E3B6E040E555DD8A4010E76
:102530003B160A0E555DD8A4010E3B16140E555DD0
:10254000D8A4010E3B16000103E00301040E556FF1
:102550000001FFEC43F09B3123E30EEC00F0800E12
:10256000016E19EC00F0120EF76EC40EF66E3BEC25
:1025700001F0800E016EC00E19EC00F0120EF76E25
:10258000DA0EF66E3BEC01F08EC329F08DC328F015
:102590008CC327F08BC326F0010EA7EC00F026D0E9
:1025A000840E026E020E086E840E036E010E046E1F
:1025B000050E096EED51136EEFEC01F0E851136E4C
:1025C000EFEC01F0F251136EEFEC01F0E651136EF7
:1025D000EFEC01F0F051136EEFEC01F0E851136EE7
:1025E000EFEC01F096948D8496948D94120EF76E14
:1025F000EC0EF66EB3EC01F0040E016E8EC329F002
:102600008DC328F08CC327F08BC326F0010EA7ECF6
:1026100000F00D0EBBEC01F00A0EBBEC01F04BC05C
:1026200057F04AC056F04DC059F04CC058F0030165
:102630005551B40DF3CFC4F0F4CFC5F05551680D2A
:10264000F3CFC6F0F4CFC7F00001C72766510301EE
:102650005503F4CFC9F0F3CFC8F055510A0DF3CFAD
:10266000CAF0F4CFCBF05551640DF3CFCCF0F4CFDA
:10267000CDF055511E0DF3CFD0F0F4CFD1F0555120
:10268000320DF3CFCEF0F4CFCFF055510F0DF3CF85
:10269000D2F0F4CFD3F042944296429042924DC091
:1026A00049F04CC048F000019A51E8BA01D0938E2D
:1026B000070E186ED00E19EC02F001EE47F0EF6A2B
:1026C00000EEF6F0EF6A449CCBEC40F0ABA206D0F3
:1026D000AB98AB880301892B000E8A230001ABA4C1
:1026E00004D0AECFA9F003018A2B0001010E42B441
:1026F000000E3B6E010E42B0000E3B16D8B454D013
:1027000080BC28D081A604D093968A9652EC44F0DF
:102710004590458293988A8880BC1CD0CBEC40F0D1
:10272000B3EC26F04A50565C136E4B505758146E5B
:102730000AEC03F00B6E14C00CF0D2510B5CD351B9
:102740000C580C50D319D8B0800A03E742849596F0
:102750008C86E2D780BE28D081A804D093988A982E
:1027600052EC44F04580459293968A8680BE1CD0F8
:10277000CBEC40F0B3EC26F04A50565C136E4B5055
:102780005758146E0AEC03F00B6E14C00CF0D251C3
:102790000B5CD3510C580C50D319D8B0800A03E706
:1027A000428495968C86E2D7000E42B4010E3B6EB1
:1027B000000E42B0010E3B1227E0010E80BC000E5D
:1027C0003B6E010E80BE000E3B12010E82B2000E67
:1027D0003B1219E093968A9693988A984294429075
:1027E000449C010E80BC000E3B6E010E80BE000EAC
:1027F0003B12010E82B2000E3B1205E0CBEC40F022
:10280000B3EC26F0EED704D093968A9693988A98E4
:102810009A51E8B27FD0010E42B6000E3B6E010E17
:1028200042B2000E3B16D8B454D082B428D081AC4A
:1028300004D0939C8A9C52EC44F045964584939A2C
:102840008A8A82B41CD0CBEC40F0B3EC26F04C501A
:10285000585C136E4D505958146E0AEC03F00B6E11
:1028600014C00CF0CA510B5CCB510C580C50CB1956
:10287000D8B0800A03E7428695968C86E2D782B666
:1028800028D081AA04D0939A8A9A52EC44F04586C3
:102890004594939C8A8C82B61CD0CBEC40F0B3EC70
:1028A00026F04C50585C136E4D505958146E0AEC7B
:1028B00003F00B6E14C00CF0CA510B5CCB510C58DA
:1028C0000C50CB19D8B0800A03E7428695968C86C7
:1028D000E2D7000E42B6010E3B6E000E42B2010E70
:1028E0003B1214E0010E82B4000E3B6E010E82B664
:1028F000000E3B12010E82B2000E3B1206E0939CCA
:102900008A9C939A8A9A4296429204D0939C8A9C7B
:10291000939A8A9A6F514A5C4E6E70514B584F6E23
:1029200071514C5C506E72514D58516E42A426D07C
:10293000000E45B0010E3B6EC6514E5CC7514F585C
:102940004F50C719D8B0800A02E6000E01D0010E20
:102950003B1603E093968A964294000E45B2010E10
:102960003B6E4FBE05D04E504F1002E0000E01D01E
:10297000010E3B1603E093988A98429442A626D013
:10298000000E45B4010E3B6EC851505CC951515800
:102990005150C919D8B0800A02E6000E01D0010ECC
:1029A0003B1603E0939A8A9A4296000E45B6010EB2
:1029B0003B6E51BE05D05050511002E0000E01D0C8
:1029C000010E3B1603E0939C8A9C429682A2ABECDC
:1029D0002CF0000E42B4010E3B6E000E42B6010E0A
:1029E0003B1201E0449C010E42B4000E3B6E010E0E
:1029F00042B6000E3B16010E42B0000E3B16010E11
:102A000042B2000E3B1602E095968C9642BC828044
:102A100042AC8290B3EC26F0000E82B6010E3B6E03
:102A2000000E82B4010E3B1604E04DC059F04CC0BC
:102A300058F0000E80BC010E3B6E000E80BE010EF1
:102A40003B1604E04BC057F04AC056F0000E44BCA1
:102A5000010E3B6E000E42BC010E3B1618E0AB535C
:102A600016E0146AABC013F0186A460E176E68ECD5
:102A700002F01CC00CF01BC00BF00C500B1002E15C
:102A800087EC40F0AB07010E18EC02F0E8D7000E1F
:102A900044BC010E3B6E010E82B0000E3B16D8B452
:102AA00092EF25F0449CF651B16F240EB15D04E124
:102AB000E1EC38F08EEF25F0570EB15DD8A47BD055
:102AC000FA510B6E200E0B5CD8A473D001EE98F077
:102AD00010EEF6F0060EF36E030E35EC03F0EF6A1F
:102AE00004EE15F011EE98F0060E2EEC03F010EC4B
:102AF0004BF0AEC3B3F0ADC3B2F0B351E8AE02D009
:102B0000000E01D0010E3B6EB351E8BE07D0B353A7
:102B100003E1B251B40802E2000E01D0010E3B16EF
:102B20000001D8B444D0B3C094F3B2C093F39FEC87
:102B300044F096C349F095C348F001EE98F010EECA
:102B4000F6F0020EF36E030E35EC03F0EF6A04EEBE
:102B500015F011EE98F0060E2EEC03F010EC4BF091
:102B6000AEC3B3F0ADC3B2F0B351E8AE02D0000EC5
:102B700001D0010E3B6EB351E8BE09D0010EB35D2A
:102B800006E303E1690EB25D02E3000E01D0010E1F
:102B90003B1600010CE0B3C090F3B2C08FF363ECBE
:102BA00044F092C347F091C346F087EC40F0429462
:102BB00042968EEF25F04D0EB15DD8A488D0F75126
:102BC0000B6E520E0B5C0FE187EC40F081A804D035
:102BD00093988A9852EC44F04580459293968A8661
:102BE0004284429072D04C0E0B5C0FE187EC40F0B7
:102BF00081A604D093968A9652EC44F04590458283
:102C000093988A884284429060D0550E0B5C0FE105
:102C100087EC40F081AC04D0939C8A9C52EC44F049
:102C200045964584939A8A8A428642924ED0440EB3
:102C30000B5C0FE187EC40F081AA04D0939A8A9A4A
:102C400052EC44F045864594939C8A8C428642928D
:102C50003CD001EE98F010EEF6F0020EF36E030E8B
:102C600035EC03F0EF6A04EE15F011EE98F0060E65
:102C70002EEC03F010EC4BF0AEC3B3F0ADC3B2F0EA
:102C8000B351E8AE02D0000E01D0010E3B6EB3513D
:102C9000E8BE09D0010EB35D06E303E1690EB25D43
:102CA00002E3000E01D0010E3B1600010EE0B3C09E
:102CB00090F3B2C08FF363EC44F092C347F091C33A
:102CC00046F087EC40F0428042948EEF25F04B0EA8
:102CD000B15D3CE101EE98F010EEF6F0020EF36EFD
:102CE000030E35EC03F0EF6A04EE15F011EE98F0E8
:102CF000060E2EEC03F010EC4BF0AEC3B3F0ADC3F8
:102D0000B2F0B351E8AE02D0000E01D0010E3B6E1E
:102D1000B351E8BE07D0B35303E1B251B40802E2A5
:102D2000000E01D0010E3B1600010EE0B3C094F37B
:102D3000B2C093F39FEC44F096C349F095C348F0BA
:102D400087EC40F0428242968EEF25F0520EB15D44
:102D500010E187EC40F081A804D093988A9852EC57
:102D600044F04580459293968A86428442908EEF45
:102D700025F04C0EB15D10E187EC40F081A604D047
:102D800093968A9652EC44F04590458293988A88AF
:102D9000428442908EEF25F0550EB15D10E187EC34
:102DA00040F081AC04D0939C8A9C52EC44F0459650
:102DB0004584939A8A8A428642928EEF25F0440E89
:102DC000B15D10E187EC40F081AA04D0939A8A9A11
:102DD00052EC44F045864594939C8A8C42864292FC
:102DE0008EEF25F0530EB15D24E1F7510B6E410ECD
:102DF0000B5C07E193968A9693988A984290429446
:102E000016D0450E0B5C07E1939A8A9A939C8A9C94
:102E1000429242960CD093968A9693988A98939A67
:102E20008A9A939C8A9C42904292429442968EEF58
:102E300025F0410EB15DD8A49AD0F7510B6E5A0E11
:102E40000B5CD8A48CD001EE98F010EEF6F0030ED7
:102E5000F36E35EC03F0EF6A04EE15F011EE98F026
:102E6000060E2EEC03F010EC4BF0AEC3B3F0ADC386
:102E7000B2F0B351E8AE02D0000E01D0010E3B6EAD
:102E8000B351E8BE09D0010EB35D06E303E1690E5C
:102E9000B25D02E3000E01D0010E3B160001D8B472
:102EA0005DD0B3C090F3B2C08FF363EC44F092C333
:102EB00047F091C346F0FD510B6E200E0B5C010EE6
:102EC000D8A4000E3B6EFE510B6E450E0B5C010E3E
:102ED000D8A4000E3B16FF510B6E4C0E0B5C010E7E
:102EE000D8A4000E3B1636E001EE98F010EEF6F096
:102EF0000B0EF36E030E35EC03F0EF6A04EE15F0E3
:102F000011EE98F0060E2EEC03F010EC4BF0AEC371
:102F1000B3F0ADC3B2F0B351E8AE02D0000E01D0B1
:102F2000010E3B6EB351E8BE07D0B35303E1B2517B
:102F3000B40802E2000E01D0010E3B1600010AE0C7
:102F4000B3C094F3B2C093F39FEC44F096C349F03E
:102F500095C348F04294429687EC40F006D0939691
:102F60008A9693988A98429042948EEF25F0450E67
:102F7000B15DD8A447D0F7510B6E4C0E0B5C3AE113
:102F800001EE98F010EEF6F0030EF36E35EC03F060
:102F9000EF6A04EE15F011EE98F0060E2EEC03F039
:102FA00010EC4BF0AEC3B3F0ADC3B2F0B351E8AE2A
:102FB00002D0000E01D0010E3B6EB351E8BE07D027
:102FC000B35303E1B251B40802E2000E01D0010E86
:102FD0003B1600010EE0B3C094F3B2C093F39FEC34
:102FE00044F096C349F095C348F04282429687EC7C
:102FF00040F006D0939A8A9A939C8A9C4292429679
:103000008EEF25F0430EB15DD8A4BED0F7510B6E04
:10301000320E0B5CD8A473D09A51E8B435D02B0E85
:10302000BBEC01F0300EBBEC01F0040E016E030EA0
:10303000076E4FC022F04EC021F055C31BF01C6A32
:103040007FEC02F01B6E14C01CF06FEC00F02B0E36
:10305000BBEC01F0300EBBEC01F0030E076E51C06B
:1030600022F050C021F055C31BF01C6A7FEC02F027
:103070001B6E14C01CF06FEC00F00D0EBBEC01F0E9
:103080000A0EBBEC01F03AD0410EBBEC01F05A0E37
:10309000BBEC01F03D0EBBEC01F0040E016E030E23
:1030A000076E4FC022F04EC021F055C31BF01C6AC2
:1030B0007FEC02F01B6E14C01CF06FEC00F0450EAC
:1030C000BBEC01F04C0EBBEC01F03D0EBBEC01F093
:1030D000030E076E51C022F050C021F055C31BF003
:1030E0001C6A7FEC02F01B6E14C01CF06FEC00F049
:1030F0000D0EBBEC01F00A0EBBEC01F043D09A516F
:10310000E8B41FD02B0EBBEC01F0300EBBEC01F08D
:10311000040E016E030E076E4FC022F04EC021F068
:1031200055C31BF01C6A7FEC02F01B6E14C01CF030
:103130006FEC00F00D0EBBEC01F00A0EBBEC01F0E1
:1031400021D0410EBBEC01F05A0EBBEC01F03D0E5C
:10315000BBEC01F0040E016E030E076E4FC022F0AF
:103160004EC021F055C31BF01C6A7FEC02F01B6EB1
:1031700014C01CF06FEC00F00D0EBBEC01F00A0E59
:10318000BBEC01F08EEF25F0420EB15D45E19A51A6
:10319000E8B41FD02B0EBBEC01F0300EBBEC01F0FD
:1031A000040E016E030E076E51C022F050C021F0D4
:1031B00055C31BF01C6A7FEC02F01B6E14C01CF0A0
:1031C0006FEC00F00D0EBBEC01F00A0EBBEC01F051
:1031D00021D0450EBBEC01F04C0EBBEC01F03D0ED6
:1031E000BBEC01F0040E016E030E076E51C022F01D
:1031F00050C021F055C31BF01C6A7FEC02F01B6E1F
:1032000014C01CF06FEC00F00D0EBBEC01F00A0EC8
:10321000BBEC01F08EEF25F0560EB15D3AE1F751AF
:103220000B6E450E0B5C1AE1560EBBEC01F0450E21
:10323000BBEC01F0040E016E8EC329F08DC328F0A3
:103240008CC327F08BC326F0010EA7EC00F00D0E07
:10325000BBEC01F00A0EBBEC01F019D0130EF76EB7
:103260000A0EF66EB3EC01F0040E016E8EC329F067
:103270008DC328F08CC327F08BC326F0010EA7EC7A
:1032800000F00D0EBBEC01F00A0EBBEC01F08EEF6E
:1032900025F0500EB15DD8A403D1F7510B6E3F0E4F
:1032A0000B5C3BE1130EF76E140EF66EB3EC01F0FF
:1032B000040E016E030E076E68C022F067C021F095
:1032C00055C31BF01C6A7FEC02F01B6E14C01CF08F
:1032D0006FEC00F0200EBBEC01F0450EBBEC01F0F2
:1032E0004C0EBBEC01F03D0EBBEC01F0030E076E83
:1032F0006AC022F069C021F055C31BF01C6A7FEC44
:1033000002F01B6E14C01CF06FEC00F00D0EBBEC55
:1033100001F00A0EBBEC01F0C1D0F7510B6E210E8B
:103320000B5C1BE14BC068F04AC067F04DC06AF00F
:103330004CC069F0AA6A040EA96E6751D3EC01F083
:103340006851D3EC01F0AA6A060EA96E6951D3EC5C
:1033500001F06A51D3EC01F0A1D0F7510301BD6F28
:103360000001DFEC4BF045AE8DD001EE98F010EE91
:10337000F6F0020EF36E030E35EC03F0EF6A04EE86
:1033800015F011EE98F0060E2EEC03F010EC4BF059
:10339000AEC3B3F0ADC3B2F0B351E8BE09D0010E75
:1033A000B35D06E303E1690EB25D02E3000E01D0F6
:1033B000010E3B6E0001B351E8AE02D0000E01D009
:1033C000010E3B1614E0B25103015503F3CF67F031
:1033D000F4CF68F00001B35103015503F35000012D
:1033E0006827030155AF03D00001B251685F0001A7
:1033F00001EE98F010EEF6F0060EF36E030E35ECCB
:1034000003F0EF6A04EE15F011EE98F0060E2EECC4
:1034100003F010EC4BF0AEC3B3F0ADC3B2F0B35158
:10342000E8BE2FD0B3BF05D0B35118E1B50EB25DE1
:1034300015E20001B25103015503F3CF69F0F4CF57
:103440006AF00001B35103015503F35000016A27EC
:10345000030155AF03D00001B2516A5F0001AA6AAF
:10346000040EA96E6751D3EC01F06851D3EC01F062
:10347000AA6A060EA96E6951D3EC01F06A51D3EC29
:1034800001F00CD068C047F067C046F06AC049F050
:1034900069C048F042804282429442968EEF25F005
:1034A0004F0EB15DD8A496D0F7510B6E3F0E0B5C5A
:1034B0001EE1130EF76E200EF66EB3EC01F0040E53
:1034C000016E076A70C022F06FC021F055C31BF077
:1034D0001C6A7FEC02F01B6E14C01CF06FEC00F055
:1034E0000D0EBBEC01F00A0EBBEC01F071D0F751F0
:1034F0000B6E210E0B5C16E1AA6A080EA96E4A50EB
:10350000D3EC01F04B50D3EC01F0130EF76E320EFA
:10351000F66EB3EC01F00D0EBBEC01F00A0EBBEC45
:1035200001F056D001EE98F010EEF6F0020EF36EB8
:10353000030E35EC03F0EF6A04EE15F011EE98F08F
:10354000060E2EEC03F010EC4BF0AEC3B3F0ADC39F
:10355000B2F0B351E8AE02D0000E01D0010E3B6EC6
:10356000B351E8BE07D0B35303E1B251320802E2CF
:10357000000E01D0010E3B1600012AE0B2510301FA
:103580005503F3CF6FF0F4CF70F00001B351030196
:103590005503F35000017027030155AF03D000011C
:1035A000B251705FAA6A080EA96E00016F51D3EC88
:1035B00001F07051D3EC01F0130EF76E320EF66E7F
:1035C000B3EC01F00D0EBBEC01F00A0EBBEC01F008
:1035D0008EEF25F0470EB15DD8A47BD0F7510B6E6E
:1035E0003F0E0B5C1EE1130EF76E480EF66EB3EC49
:1035F00001F0040E016E076A72C022F071C021F062
:1036000055C31BF01C6A7FEC02F01B6E14C01CF04B
:103610006FEC00F00D0EBBEC01F00A0EBBEC01F0FC
:1036200056D001EE98F010EEF6F0020EF36E030E97
:1036300035EC03F0EF6A04EE15F011EE98F0060E8B
:103640002EEC03F010EC4BF0AEC3B3F0ADC3B2F010
:10365000B351E8AE02D0000E01D0010E3B6EB35163
:10366000E8BE07D0B35303E1B2511E0802E2000ED8
:1036700001D0010E3B1600012AE0B25103015503AF
:10368000F3CF71F0F4CF72F00001B3510301550391
:10369000F35000017227030155AF03D00001B2516E
:1036A000725FAA6A0A0EA96E00017151D3EC01F093
:1036B0007251D3EC01F0130EF76E5C0EF66EB3ECA4
:1036C00001F00D0EBBEC01F00A0EBBEC01F08EEF29
:1036D00025F0480EB15D04E03F0EB15DD8A442D2A2
:1036E000130EF76E740EF66EB3EC01F00D0EBBEC1C
:1036F00001F00A0EBBEC01F0130EF76E9E0EF66E93
:10370000B3EC01F00D0EBBEC01F00A0EBBEC01F0C6
:10371000130EF76EAC0EF66EB3EC01F00D0EBBECB3
:1037200001F00A0EBBEC01F0130EF76EC40EF66E3C
:10373000B3EC01F00D0EBBEC01F00A0EBBEC01F096
:10374000130EF76EDC0EF66EB3EC01F00D0EBBEC53
:1037500001F00A0EBBEC01F0130EF76EF40EF66EDC
:10376000B3EC01F00D0EBBEC01F00A0EBBEC01F066
:10377000140EF76E100EF66EB3EC01F00D0EBBECEE
:1037800001F00A0EBBEC01F0140EF76E2C0EF66E73
:10379000B3EC01F00D0EBBEC01F00A0EBBEC01F036
:1037A000140EF76E500EF66EB3EC01F00D0EBBEC7E
:1037B00001F00A0EBBEC01F0140EF76E7A0EF66EF5
:1037C000B3EC01F00D0EBBEC01F00A0EBBEC01F006
:1037D000140EF76EA80EF66EB3EC01F00D0EBBECF6
:1037E00001F00A0EBBEC01F0140EF76ECC0EF66E73
:1037F000B3EC01F00D0EBBEC01F00A0EBBEC01F0D6
:10380000140EF76EE60EF66EB3EC01F00D0EBBEC87
:1038100001F00A0EBBEC01F0150EF76E060EF66E07
:10382000B3EC01F00D0EBBEC01F00A0EBBEC01F0A5
:10383000150EF76E140EF66EB3EC01F00D0EBBEC28
:1038400001F00A0EBBEC01F0150EF76E280EF66EB5
:10385000B3EC01F00D0EBBEC01F00A0EBBEC01F075
:10386000150EF76E4A0EF66EB3EC01F00D0EBBECC2
:1038700001F00A0EBBEC01F0150EF76E680EF66E45
:10388000B3EC01F00D0EBBEC01F00A0EBBEC01F045
:10389000150EF76E7A0EF66EB3EC01F00D0EBBEC62
:1038A00001F00A0EBBEC01F0150EF76EA60EF66ED7
:1038B000B3EC01F00D0EBBEC01F00A0EBBEC01F015
:1038C000150EF76ED00EF66EB3EC01F00D0EBBECDC
:1038D00001F00A0EBBEC01F0150EF76EF60EF66E57
:1038E000B3EC01F00D0EBBEC01F00A0EBBEC01F0E5
:1038F000160EF76E200EF66EB3EC01F00D0EBBEC5B
:1039000001F00A0EBBEC01F0160EF76E340EF66EE7
:10391000B3EC01F00D0EBBEC01F00A0EBBEC01F0B4
:10392000160EF76E440EF66EB3EC01F00D0EBBEC06
:1039300001F00A0EBBEC01F0160EF76E5C0EF66E8F
:10394000B3EC01F00D0EBBEC01F00A0EBBEC01F084
:10395000160EF76E860EF66EB3EC01F00D0EBBEC94
:1039600001F00A0EBBEC01F0160EF76E9E0EF66E1D
:10397000B3EC01F00D0EBBEC01F00A0EBBEC01F054
:10398000160EF76ECA0EF66EB3EC01F00D0EBBEC20
:1039900001F00A0EBBEC01F0160EF76EE80EF66EA3
:1039A000B3EC01F00D0EBBEC01F00A0EBBEC01F024
:1039B000170EF76E0A0EF66EB3EC01F00D0EBBECAF
:1039C00001F00A0EBBEC01F0170EF76E280EF66E32
:1039D000B3EC01F00D0EBBEC01F00A0EBBEC01F0F4
:1039E000170EF76E340EF66EB3EC01F00D0EBBEC55
:1039F00001F00A0EBBEC01F0170EF76E680EF66EC2
:103A0000B3EC01F00D0EBBEC01F00A0EBBEC01F0C3
:103A1000170EF76E820EF66EB3EC01F00D0EBBECD6
:103A200001F00A0EBBEC01F0170EF76E960EF66E63
:103A3000B3EC01F00D0EBBEC01F00A0EBBEC01F093
:103A4000170EF76EBE0EF66EB3EC01F00D0EBBEC6A
:103A500001F00A0EBBEC01F0170EF76ED00EF66EF9
:103A6000B3EC01F00D0EBBEC01F00A0EBBEC01F063
:103A7000170EF76EF80EF66EB3EC01F00D0EBBEC00
:103A800001F00A0EBBEC01F0180EF76E300EF66E68
:103A9000B3EC01F00D0EBBEC01F00A0EBBEC01F033
:103AA000180EF76E4E0EF66EB3EC01F00D0EBBEC79
:103AB00001F00A0EBBEC01F0180EF76E700EF66EF8
:103AC000B3EC01F00D0EBBEC01F00A0EBBEC01F003
:103AD000180EF76E900EF66EB3EC01F00D0EBBEC07
:103AE00001F00A0EBBEC01F0180EF76EA80EF66E90
:103AF000B3EC01F00D0EBBEC01F00A0EBBEC01F0D3
:103B0000180EF76EC20EF66EB3EC01F00D0EBBECA4
:103B100001F00A0EBBEC01F0180EF76EE00EF66E27
:103B2000B3EC01F00D0EBBEC01F00A0EBBEC01F0A2
:103B3000180EF76EFE0EF66EB3EC01F00D0EBBEC38
:103B400001F00A0EBBEC01F0190EF76E260EF66EB0
:103B5000B3EC01F00D0EBBEC01F00A0EBBEC01F072
:103B60008EEF25F04E0EB15D37E1000E9BB1010ED8
:103B7000010AD8B49B91D8A49B81190EF76E500E00
:103B8000F66EB3EC01F09B3110E34C0EBBEC01F090
:103B9000430EBBEC01F0440EBBEC01F00D0EBBEC90
:103BA00001F00A0EBBEC01F00FD04C0EBBEC01F0A3
:103BB000450EBBEC01F0440EBBEC01F00D0EBBEC6E
:103BC00001F00A0EBBEC01F0AA6A1E0EA96E9B5111
:103BD000D3EC01F08EEF25F0590EB15D3CE1000E03
:103BE0009AB1010E010AD8B49A91D8A49A81450ECF
:103BF000BBEC01F0630EBBEC01F0680EBBEC01F016
:103C00006F0EBBEC01F0200EBBEC01F09A310DE31E
:103C10004F0EBBEC01F04E0EBBEC01F00D0EBBECF9
:103C200001F00A0EBBEC01F00ED04F0EBBEC01F020
:103C3000460EBBEC01F0BBEC01F00D0EBBEC01F04D
:103C40000A0EBBEC01F0AA6A0F0EA96E9A51D3ECD2
:103C500001F08EEF25F0510EB15DD8A4AAD001EE8F
:103C600098F010EEF6F0020EF36E030E35EC03F052
:103C7000EF6A190EF76E5E0EF66E01EE98F049ECE3
:103C800003F00BE10301040E556FAA6A110EA96E31
:103C90005551D3EC01F0000149D0190EF76E620EB8
:103CA000F66E01EE98F049EC03F00BE10301140EFF
:103CB000556FAA6A110EA96E5551D3EC01F000019F
:103CC00035D001EE98F0EECFF3FFEFCFF4FFF350D5
:103CD000310AF41002E0000E01D0010E3B6E190E05
:103CE000F76E660EF66E01EE98F052EC03F03B12A2
:103CF0000BE00301020E556FAA6A110EA96E555111
:103D0000D3EC01F0000112D0190EF76E6A0EF66EB8
:103D100001EE98F049EC03F009E103010A0E556F3A
:103D2000AA6A110EA96E5551D3EC01F00301555149
:103D300016EC09F035C039F034C038F033C037F034
:103D400032C036F0356A346A336A800E326E09EC5E
:103D500008F035C0AFF034C0AEF033C0ADF032C0C3
:103D6000ACF0190EF76E6E0EF66EB3EC01F0040EA9
:103D7000016EAFC029F0AEC028F0ADC027F0ACC0D6
:103D800026F0010EA7EC00F0200EBBEC01F0640E53
:103D9000BBEC01F0650EBBEC01F0670EBBEC01F073
:103DA0000D0EBBEC01F00A0EBBEC01F000018EEF32
:103DB00025F05A0EB15D41E1000E9AB7010E010ADD
:103DC000D8B49A97D8A49A87190EF76E800EF66E1B
:103DD000B3EC01F09A51E8A616D0730EBBEC01F0DB
:103DE0006F0EBBEC01F0750EBBEC01F0740EBBEC7A
:103DF00001F0680EBBEC01F00D0EBBEC01F00A0EF9
:103E0000BBEC01F012D06E0EBBEC01F06F0EBBEC00
:103E100001F0720EBBEC01F0640EBBEC01F00D0E74
:103E2000BBEC01F00A0EBBEC01F0AA6A0F0EA96E02
:103E30009A51D3EC01F08EEF25F0260EB15D23E10F
:103E40005A0E665D03E1B40E666F02D05A0E666FBD
:103E5000190EF76E920EF66EB3EC01F0040E016EC1
:103E6000030E076E66516DEC00F00D0EBBEC01F019
:103E70000A0EBBEC01F0AA6A0E0EA96E6651D3ECD5
:103E800001F08EEF25F04A0EB15DD8A494D0190E42
:103E9000F76EA80EF66EB3EC01F0F7510B6E4E0EF6
:103EA0000B5C0FE13A0EBBEC01F0200EBBEC01F015
:103EB0006F0EBBEC01F0660EBBEC01F0BBEC01F049
:103EC0009A9BF7510B6E460E0B5C08E1190EF76ECC
:103ED000B00EF66EB3EC01F09A899A8BF7510B6E27
:103EE000440E0B5C08E1190EF76EBC0EF66EB3ECD7
:103EF00001F09A999A8BF7510301BD6F0001DFEC35
:103F00004BF045AE49D001EE98F010EEF6F0020EFF
:103F1000F36E050E35EC03F0EF6A01EE98F020EC3D
:103F200000F00301856F1CC086F3190EF76ECE0EEC
:103F3000F66EB3EC01F0040E016E076A86C31CF046
:103F400085C31BF06FEC00F0AA6A1C0EA96E86C335
:103F500014F085C313F0186A0A0E176E68EC02F0AD
:103F6000266E14C027F02650D3EC01F02750D3EC76
:103F700001F0166A070E156EA10E146E200E136E58
:103F800085C31BF086C31CF01D6A1E6A3DEC02F05F
:103F900014C084F313C083F300010D0EBBEC01F0D9
:103FA0000A0EBBEC01F0AA6A0F0EA96E9A51D3EC6F
:103FB00001F08EEF25F0540EB15DD8A4AED0F751CC
:103FC0000301BD6F0001DFEC4BF045AEA3D001EE65
:103FD00098F010EEF6F0020EF36E050E35EC03F0DD
:103FE000EF6A01EE98F020EC00F08A6F1CC08BF0B5
:103FF000190EF76EDC0EF66EB3EC01F0040E016ED6
:10400000076A8BC01CF08AC01BF06FEC00F00D0E2D
:10401000BBEC01F00A0EBBEC01F0190EF76EEE0ED0
:10402000F66EB3EC01F00D0EBBEC01F00A0EBBEC2A
:1040300001F0B951120AC00ED8B4B81902E1000E4D
:1040400001D0010E3B6EB951250A800ED8B4B819C3
:1040500002E1000E01D0010E3B16B9514B0AB81116
:1040600002E1000E01D0010E3B16B951960AB811BB
:1040700002E1000E01D0010E3B16B951E10AB81160
:1040800002E1000E01D0010E3B160CE01A0EF76E95
:10409000180EF66EB3EC01F00D0EBBEC01F00A0E3B
:1040A000BBEC01F0AA6A1F0EA96E8A51D3EC01F095
:1040B0008B51D3EC01F01A0EF76E620EF66EB3EC74
:1040C00001F00D0EBBEC01F00A0EBBEC01F00B0E83
:1040D000086EB80E026E94EC01F01CE3A96FA99B68
:1040E0009A3103E3A951BBEC01F0590EA95D12E12D
:1040F0001A0EF76E840EF66EB3EC01F00D0EBBECEB
:1041000001F00A0EBBEC01F08BC0B9F08AC0B8F028
:10411000FFEC43F0B16B8EEF25F0250EB15D38E179
:10412000000E9AB3010E010AD8B49A93D8A49A83C8
:104130001A0EF76E9C0EF66EB3EC01F09A51E8B2CF
:104140000DD04F0EBBEC01F04E0EBBEC01F00D0E8E
:10415000BBEC01F00A0EBBEC01F00ED04F0EBBEC35
:1041600001F0460EBBEC01F0BBEC01F00D0EBBEC18
:1041700001F00A0EBBEC01F0800E016E10EC00F0B5
:10418000AA6A0F0EA96E9A51D3EC01F08EEF25F0BA
:104190002A0EB15D38E101EE98F010EEF6F0020E55
:1041A000F36E030E35EC03F0EF6A04EE15F011EE3A
:1041B00098F0060E2EEC03F010EC4BF0AEC3B3F00B
:1041C000ADC3B2F0B351E8AE02D0000E01D0010E83
:1041D0003B6EB351E8BE07D0B35303E1B2515A0866
:1041E00002E2000E01D0010E3B16000109E0B2C050
:1041F00059F3AA6A100EA96E03015951D3EC01F0CC
:1042000000018EEF25F0460EB15DD8A49FD0F75186
:104210000B6E3F0E0B5C30E16F51735D266E70517B
:104220007459276E27C022F026C021F055C31BF019
:104230001C6A7FEC02F0906F14C091F09A51E8A6CE
:1042400004D0B40E905F000E915B1A0EF76EAA0EAA
:10425000F66EB3EC01F0040E016E030E076E91C012
:104260001CF090C01BF06FEC00F00D0EBBEC01F0E9
:104270000A0EBBEC01F068D0F7510301BD6F0001DD
:10428000DFEC4BF045AE42D001EE98F010EEF6F0C8
:10429000020EF36E030E35EC03F0EF6A04EE15F038
:1042A00011EE98F0060E2EEC03F010EC4BF0AEC3BE
:1042B000B3F0ADC3B2F0B351E8BE27D0B251B311E1
:1042C00024E0B3C074F0B2C073F09A51E8A604D0F1
:1042D000B40E7327000E7423735103015503F3CFFB
:1042E00026F0F4CF27F00001745103015503F35079
:1042F000272655AF03D000017351275E00016F518F
:104300002624736F70512720746F09D0F7510B6EFC
:10431000210E0B5C04E14BC074F04AC073F0AA6A32
:104320000C0EA96E7351D3EC01F07451D3EC01F073
:104330001A0EF76EC00EF66EB3EC01F00D0EBBEC6C
:1043400001F00A0EBBEC01F08EEF25F0230EB15DFB
:104350002CE1000E9AB5010E010AD8B49A95D8A4A2
:104360009A851A0EF76ECC0EF66EB3EC01F09A51E8
:10437000E8B40AD0410EBBEC01F00D0EBBEC01F02D
:104380000A0EBBEC01F009D0420EBBEC01F00D0EA1
:10439000BBEC01F00A0EBBEC01F0AA6A0F0EA96E8D
:1043A0009A51D3EC01F08EEF25F0490EB15DD8A4FF
:1043B00097EF24F00D0EBBEC01F00A0EBBEC01F000
:1043C0001A0EF76ED80EF66EB3EC01F00D0EBBECC4
:1043D00001F00A0EBBEC01F01A0EF76EFA0EF66E43
:1043E000B3EC01F0040E016E076A70C022F06FC0DA
:1043F00021F055C31BF01C6A7FEC02F01B6E14C049
:104400001CF06FEC00F0200EBBEC01F0640EBBEC76
:1044100001F0650EBBEC01F0670EBBEC01F00D0E78
:10442000BBEC01F00A0EBBEC01F01B0EF76E0E0E9A
:10443000F66EB3EC01F0040E016E076A72C022F052
:1044400071C021F055C31BF01C6A7FEC02F01B6E9B
:1044500014C01CF06FEC00F0200EBBEC01F0640EF9
:10446000BBEC01F0650EBBEC01F0670EBBEC01F09C
:104470000D0EBBEC01F00A0EBBEC01F06F51735D49
:10448000266E70517459276E27C022F026C021F085
:1044900055C31BF01C6A7FEC02F0906F14C091F0C2
:1044A0009A51E8A604D0B40E905F000E915B1B0EEB
:1044B000F76E240EF66EB3EC01F0040E016E076A7F
:1044C00091C01CF090C01BF06FEC00F0200EBBEC14
:1044D00001F0640EBBEC01F0650EBBEC01F0670E61
:1044E000BBEC01F00D0EBBEC01F00A0EBBEC01F0D1
:1044F0001B0EF76E420EF66EB3EC01F0040E016E69
:1045000066516CEC00F0200EBBEC01F0640EBBECCD
:1045100001F0650EBBEC01F0670EBBEC01F00D0E77
:10452000BBEC01F00A0EBBEC01F01B0EF76E620E45
:10453000F66EB3EC01F0040E016E030159516CEC00
:1045400000F0200EBBEC01F0640EBBEC01F0650E38
:10455000BBEC01F0670EBBEC01F00D0EBBEC01F003
:104560000A0EBBEC01F01B0EF76E840EF66EB3EC78
:1045700001F000019A51E8A209D04F0EBBEC01F006
:10458000460EBBEC01F0BBEC01F006D04F0EBBECCD
:1045900001F04E0EBBEC01F00D0EBBEC01F00A0E6B
:1045A000BBEC01F01B0EF76E980EF66EB3EC01F04B
:1045B000040E016E030E076E68C022F067C021F082
:1045C00055C31BF01C6A7FEC02F01B6E14C01CF07C
:1045D0006FEC00F0200EBBEC01F0450EBBEC01F0DF
:1045E0004C0EBBEC01F03A0EBBEC01F0200EBBEC24
:1045F00001F0030E076E6AC022F069C021F055C3B6
:104600001BF01C6A7FEC02F01B6E14C01CF06FECF8
:1046100000F00D0EBBEC01F00A0EBBEC01F01A0E1F
:10462000F76ECC0EF66EB3EC01F09A51E8B404D0FC
:10463000410EBBEC01F003D0420EBBEC01F00D0EBD
:10464000BBEC01F00A0EBBEC01F01B0EF76EA80EDE
:10465000F66EB3EC01F09A51E8B60DD04E0EBBECFD
:1046600001F06F0EBBEC01F0720EBBEC01F0640EBA
:10467000BBEC01F00FD0530EBBEC01F06F0EBBECA6
:1046800001F0750EBBEC01F0740EBBEC01F0680E8E
:10469000BBEC01F00D0EBBEC01F00A0EBBEC01F01F
:1046A000190EF76EDC0EF66EB3EC01F0040E016E1F
:1046B000076AB9C01CF0B8C01BF06FEC00F00D0E1B
:1046C000BBEC01F00A0EBBEC01F01B0EF76EB80E4E
:1046D000F66EB3EC01F09A3107E34F0EBBEC01F03C
:1046E0004E0EBBEC01F008D04F0EBBEC01F0460EB5
:1046F000BBEC01F0BBEC01F00D0EBBEC01F00A0EBF
:10470000BBEC01F01B0EF76EC80EF66EB3EC01F0B9
:104710009A51E8AA11D09A51E8A807D01B0EF76E5B
:10472000D20EF66EB3EC01F006D01B0EF76EDC0E67
:10473000F66EB3EC01F008D04F0EBBEC01F0460E64
:10474000BBEC01F0BBEC01F0000E9ABB010E3B6E1E
:10475000000E9AB9010E3B161EE00D0EBBEC01F0E7
:104760000A0EBBEC01F01B0EF76EEC0EF66EB3EC0E
:1047700001F0040E016E076A86C31CF085C31BF0AE
:104780006FEC00F0200EBBEC01F0480EBBEC01F02A
:104790007A0EBBEC01F00D0EBBEC01F00A0EBBEC87
:1047A00001F01C0EF76E000EF66EB3EC01F0030183
:1047B000555116EC09F035C039F034C038F033C02B
:1047C00037F032C036F0356A346A336A800E326EA2
:1047D00009EC08F035C0AFF034C0AEF033C0ADF036
:1047E00032C0ACF0040E016EAFC029F0AEC028F0AC
:1047F000ADC027F0ACC026F0010EA7EC00F0200EF3
:10480000BBEC01F0640EBBEC01F0650EBBEC01F0FB
:10481000670EBBEC01F00D0EBBEC01F00A0EBBEC19
:1048200001F01C0EF76E0C0EF66EB3EC01F00001F9
:104830009B310AE34C0EBBEC01F0430EBBEC01F0E4
:10484000440EBBEC01F009D04C0EBBEC01F0450E60
:10485000BBEC01F0440EBBEC01F00D0EBBEC01F023
:104860000A0EBBEC01F01C0EF76E1C0EF66EB3ECDC
:1048700001F0040E016E3DC329F03CC328F03BC398
:1048800027F03AC326F0050EA7EC00F01C0EF76ED9
:10489000280EF66EB3EC01F0040E016E41C329F050
:1048A00040C328F03FC327F03EC326F0050EA7EC17
:1048B00000F00D0EBBEC01F00A0EBBEC01F01C0E7B
:1048C000F76E360EF66EB3EC01F0040E016E8EC379
:1048D00029F08DC328F08CC327F08BC326F0010E7E
:1048E000A7EC00F00D0EBBEC01F00A0EBBEC01F0E2
:1048F0001C0EF76E4A0EF66EB3EC01F0040E016E5C
:10490000076A8AC31BF01C6A6FEC00F01C0EF76E7E
:10491000520EF66EB3EC01F0076A89C31BF01C6AF5
:104920006FEC00F0000EBBEC01F0B16BF7D03C0E69
:10493000B15D36E11C0EF76E5A0EF66EB3EC01F067
:104940000D0EBBEC01F00A0EBBEC01F0AEEC01F079
:10495000A96FA99B9A3103E3A951BBEC01F0590E51
:10496000A95D1DE18FEC37F042BE0DD01C0EF76E35
:10497000680EF66EB3EC01F00D0EBBEC01F00A0E02
:10498000BBEC01F00CD01C0EF76E7E0EF66EB3EC95
:1049900001F00D0EBBEC01F00A0EBBEC01F0BED035
:1049A0005E0EB15D36E11C0EF76E5A0EF66EB3EC7C
:1049B00001F00D0EBBEC01F00A0EBBEC01F0AEEC09
:1049C00001F0A96FA99B9A3103E3A951BBEC01F057
:1049D000590EA95D1DE137EC38F043B00DD01C0E27
:1049E000F76E980EF66EB3EC01F00D0EBBEC01F015
:1049F0000A0EBBEC01F00CD01C0EF76EB00EF66E7A
:104A0000B3EC01F00D0EBBEC01F00A0EBBEC01F0B3
:104A100085D05B0EB15D35E101EE98F010EEF6F059
:104A2000020EF36E080E35EC03F0EF6A04EE1CF094
:104A300011EE98F0140E2EEC03F034EC4BF0B3C3EF
:104A40003DF3B2C33CF3B1C33BF3B0C33AF31C0E26
:104A5000F76ECC0EF66EB3EC01F0040E016E3DC3A2
:104A600029F03CC328F03BC327F03AC326F0050EDB
:104A7000A7EC00F00D0EBBEC01F00A0EBBEC01F050
:104A80004DD05D0EB15D35E101EE98F010EEF6F01F
:104A9000020EF36E090E35EC03F0EF6A04EE1CF023
:104AA00011EE98F0140E2EEC03F034EC4BF0B3C37F
:104AB00041F3B2C340F3B1C33FF3B0C33EF31C0EA6
:104AC000F76ED80EF66EB3EC01F0040E016E41C322
:104AD00029F040C328F03FC327F03EC326F0050E5F
:104AE000A7EC00F00D0EBBEC01F00A0EBBEC01F0E0
:104AF00015D09A3113E33F0EBBEC01F03E0EBBEC38
:104B000001F000EEF6F0EE5003E0BBEC01F0FBD755
:104B10000D0EBBEC01F00A0EBBEC01F000EEF6F05E
:104B2000EF6AB16B42BC1DD16F514A5C4E6E705141
:104B30004B584F6E71514C5C506E72514D58516EC6
:104B4000000E45B0010E3B6EC6514E5CC7514F582A
:104B50004F50C719D8B0800A02E6000E01D0010EEE
:104B60003B1603E093968A96449C000E45B2010ED4
:104B70003B6E4FBE05D04E504F1002E0000E01D0EC
:104B8000010E3B1603E093988A98449C000E42B0B5
:104B9000010E3B6E010E42BE000E3B16D8B440D053
:104BA0004A505E5C4B505F584B505F18D8B0800A3B
:104BB0000CE681A604D093968A9652EC44F0459078
:104BC000458293988A8895968C865E504A5C5F50A1
:104BD0004B584B505F18D8B0800A0CE681A804D01F
:104BE00093988A9852EC44F04592458093968A8631
:104BF00095968C865F504B5C03E15E504A5C02E008
:104C0000000E01D0010E3B6E000E42BC010E3B12A5
:104C1000000106E093968A9693988A984290449C65
:104C2000010E9AB3000E3B6E49AE02D0000E01D0C9
:104C3000010E3B164850C85D4950C9594950C91921
:104C4000D8B0800A02E6000E01D0010E3B16D8B49F
:104C500075D0000E45B4010E3B6EC851505CC95171
:104C600051585150C919D8B0800A02E6000E01D03F
:104C7000010E3B1603E0939A8A9A449C000E45B6B7
:104C8000010E3B6E51BE05D05050511002E0000E97
:104C900001D0010E3B1603E0939C8A9C449C010EBC
:104CA00043B0000E3B6E000E42B2010E3B16D8B46C
:104CB00045D071514C5C506E72514D58516E5050F0
:104CC000485C5150495851504918D8B0800A0CE6F8
:104CD00081AA04D0939A8A9A52EC44F0459445866E
:104CE000939C8A8C95968C864850505C49505158BC
:104CF00051504918D8B0800A0CE681AC04D0939C7E
:104D00008A9C52EC44F045964584939A8A8A9596FB
:104D10008C864950515C03E14850505C02E0000E23
:104D200001D0010E3B6E000E42BC010E3B12000191
:104D300005E0939C8A9C939A8A9A4292010E42B40F
:104D4000000E3B6E010E42B6000E3B16010E42B045
:104D5000000E3B16010E42B2000E3B1602E0959685
:104D60008C9664EF13F06F514A5C4E6E70514B5845
:104D70004F6E71514C5C506E72514D58516E4FBE1A
:104D800002D0000E01D0010E3B6E4E50C65D4F505A
:104D9000C7594F50C719D8B0800A02E7000E01D09A
:104DA000010E3B1202E0838201D0839251BE02D0F9
:104DB000000E01D0010E3B6E5050C85D5150C959D4
:104DC0005150C919D8B0800A02E7000E01D0010E77
:104DD0003B1202E0838001D083909A51E8A614D060
:104DE000C4514E26C5514F22C6514E5CC7514F5833
:104DF0004F50C719D8B0800A06E7C6514E5C4E6EB8
:104E0000C7514F584F6E15D04FAE04D0C6514E26E5
:104E1000C7514F22C6514E5CC7514F584F50C7190A
:104E2000D8B0800A06E7C6514E5C4E6EC7514F5847
:104E30004F6E9B3102E304D802D0AAEC2AF0120094
:104E40009A51E8B2E0EF29F043B077D143BE1CD1CC
:104E5000FE0E5014526EFF0E5114536E53AE8ED090
:104E6000800E016E19EC00F0450E43EC01F04C0E83
:104E700043EC01F03A0E43EC01F0200E43EC01F05C
:104E80002D0E43EC01F053C00CF052C00BF00CAEF1
:104E900003D00B6CE86A0C56CA510B5CCB510C5812
:104EA0000C50CB19D8B0800A04E6200E43EC01F078
:104EB0001BD053C00CF052C00BF00CAE03D00B6CE7
:104EC000E86A0C560CC022F00BC021F0CBC01CF0DD
:104ED000CAC01BF07FEC02F09D6F800E016E010EC8
:104EE000076E9D516DEC00F0800E016E010E076E95
:104EF00053C00CF052C00BF00CAE03D00B6CE86A40
:104F00000C560CC022F00BC021F055C31BF01C6ADC
:104F10007FEC02F01B6E14C01CF06FEC00F02E0E44
:104F200043EC01F053C00CF052C00BF00CAE03D0B8
:104F30000B6CE86A0C560CC022F00BC021F055C374
:104F40001BF01C6A7FEC02F017C09DF09D510A0D0A
:104F5000F3CF26F0F4CF27F027C014F026C013F0CB
:104F6000186A55C317F068EC02F09D6F800E016E51
:104F7000010E076E9D516DEC00F085D0800E016E24
:104F800019EC00F0450E43EC01F04C0E43EC01F03F
:104F90003A0E43EC01F0200E43EC01F0CC51525C90
:104FA000CD5153585350CD19D8B0800A04E6200E85
:104FB00043EC01F012D053C022F052C021F0CDC01A
:104FC0001CF0CCC01BF07FEC02F09D6F800E016ED8
:104FD000010E076E9D516DEC00F0CA51525CCB5131
:104FE00053585350CB19D8B0800A04E6200E43EC36
:104FF00001F012D053C022F052C021F0CBC01CF0FF
:10500000CAC01BF07FEC02F09D6F800E016E010E96
:10501000076E9D516DEC00F0800E016E010E076E63
:1050200053C022F052C021F055C31BF01C6A7FEC24
:1050300002F01B6E14C01CF06FEC00F02E0E43EC5F
:1050400001F053C022F052C021F055C31BF01C6A7E
:105050007FEC02F017C09DF09D510A0DF3CF26F0B2
:10506000F4CF27F027C014F026C013F0186A55C3F8
:1050700017F068EC02F09D6F800E016E010E076E56
:105080009D516DEC00F058D0356A346A200E336EB5
:10509000820E326E37C339F036C338F035C337F07D
:1050A00034C336F06FEC08F0BDEC08F0526E33C03C
:1050B00053F0800E016E19EC00F0450E43EC01F048
:1050C0004C0E43EC01F03A0E43EC01F0200E43ECA1
:1050D00001F043EC01F037C335F036C334F035C38B
:1050E00033F034C332F0396A386A200E376E820EDC
:1050F000366EBFEC06F0010803E0200E43EC01F031
:10510000800E016E076A53C022F052C021F01C6A63
:105110000A0E1B6E7FEC02F01B6E14C01CF06FECCD
:1051200000F02E0E43EC01F0010E076E53C01CF090
:1051300052C01BF06FEC00F00AD0800E016E19EC2B
:1051400000F01C0EF76EE40EF66E3BEC01F08AAC3C
:1051500003D0000E43EC01F08AAA03D0010E43EC09
:1051600001F0010E8ABA000E3B6E010E8ABC000EE1
:105170003B1603E0200E43EC01F08AA803D0030E97
:1051800043EC01F08AA603D0020E43EC01F0010EBD
:105190008AB6000E3B6E010E8AB8000E3B1603E085
:1051A000200E43EC01F043BE98D042BE8FD043BEE8
:1051B00007D0FE0E4E14546EFF0E4F14556E04D0E1
:1051C00047C055F046C054F0410E43EC01F05A0E72
:1051D00043EC01F03A0E43EC01F0200E43EC01F0F9
:1051E000CC51545CCD5155585550CD19D8B0800A8A
:1051F00004E6200E43EC01F012D055C022F054C05A
:1052000021F0CDC01CF0CCC01BF07FEC02F09D6FF4
:10521000800E016E010E076E9D516DEC00F0CA51BB
:10522000545CCB5155585550CB19D8B0800A04E680
:10523000200E43EC01F012D055C022F054C021F0F2
:10524000CBC01CF0CAC01BF07FEC02F09D6F800E3B
:10525000016E010E076E9D516DEC00F0800E016E27
:10526000010E076E55C022F054C021F055C31BF04B
:105270001C6A7FEC02F01B6E14C01CF06FEC00F097
:105280002E0E43EC01F055C022F054C021F055C35E
:105290001BF01C6A7FEC02F017C09DF09D510A0DB7
:1052A000F3CF26F0F4CF27F027C014F026C013F078
:1052B000186A55C317F068EC02F09D6F800E016EFE
:1052C000010E076E9D516DEC00F006D01C0EF76EBE
:1052D000EE0EF66E3BEC01F067D0356A346A200EB4
:1052E000336E820E326E33C339F032C338F031C3BD
:1052F00037F030C336F06FEC08F0BDEC08F0546EB8
:1053000033C055F0410E43EC01F05A0E43EC01F06E
:105310003A0E43EC01F0200E43EC01F033C335F0BC
:1053200032C334F031C333F030C332F0396A386AF3
:10533000480E376E850E366EBFEC06F0010803E0AE
:10534000200E43EC01F033C335F032C334F031C3E7
:1053500033F030C332F0396A386A200E376E820E6D
:10536000366EBFEC06F0010803E0200E43EC01F0BE
:10537000800E016E076A55C022F054C021F01C6AED
:105380000A0E1B6E7FEC02F01B6E14C01CF06FEC5B
:1053900000F02E0E43EC01F0010E076E55C01CF01C
:1053A00054C01BF06FEC00F0800E016EC00E19ECC3
:1053B00000F01C0EF76EF80EF66E3BEC01F0C9D053
:1053C00042BEB2D043BE07D0FE0E4E14546EFF0E46
:1053D0004F14556E04D047C055F046C054F0800EAF
:1053E000016E19EC00F01D0EF76E0E0EF66E3BEC22
:1053F00001F0CC51545CCD5155585550CD19D8B011
:10540000800A04E6200E43EC01F012D055C022F0D1
:1054100054C021F0CDC01CF0CCC01BF07FEC02F0DA
:105420009D6F800E016E010E076E9D516DEC00F0B8
:10543000CA51545CCB5155585550CB19D8B0800A3D
:1054400004E6200E43EC01F012D055C022F054C007
:1054500021F0CBC01CF0CAC01BF07FEC02F09D6FA6
:10546000800E016E010E076E9D516DEC00F0800EF6
:10547000016E010E076E55C022F054C021F055C3D5
:105480001BF01C6A7FEC02F01B6E14C01CF06FEC6A
:1054900000F02E0E43EC01F055C022F054C021F074
:1054A00055C31BF01C6A7FEC02F017C09DF09D51A4
:1054B0000A0DF3CF26F0F4CF27F027C014F026C052
:1054C00013F0186A55C317F068EC02F09D6F800E58
:1054D000016E010E076E9D516DEC00F0200E43EC45
:1054E00001F0640E43EC01F0650E43EC01F0670E31
:1054F00043EC01F0200E43EC01F08AA803D0030E28
:1055000043EC01F08AA603D0020E43EC01F0010E39
:105510008AB6000E3B6E010E8AB8000E3B1603E001
:10552000200E43EC01F00AD0800E016E19EC00F061
:105530001D0EF76E180EF66E3BEC01F0800E016E3C
:10554000C00E19EC00F01D0EF76E2E0EF66E3BEC41
:1055500001F012000EEC00F06F514A5C4E6E70517B
:105560004B584F6E71514C5C506E72514D58516E8C
:105570009A51E8A614D0C4514E26C5514F22C651A7
:105580004E5CC7514F584F50C719D8B0800A06E734
:10559000C6514E5C4E6EC7514F584F6E15D04FAE30
:1055A00004D0C6514E26C7514F22C6514E5CC7513A
:1055B0004F584F50C719D8B0800A06E7C6514E5C05
:1055C0004E6EC7514F584F6E449A51BE448A51C0D7
:1055D0000CF050C00BF00CAE03D00B6CE86A0C560C
:1055E0000CC022F00BC021F055C31BF01C6A7FECED
:1055F00002F0626F14C063F063C014F062C013F075
:10560000020E33EC02F09C6F00EEDAF09C51EBCF0F
:105610000BF00BC0D4F063C014F062C013F0010EA5
:1056200033EC02F09C6F00EEDAF09C51EBCF0BF004
:105630000BC0D5F063C014F062C013F0000E33EC61
:1056400002F09C6F00EEDAF09C51EBCF0BF00BC038
:10565000D6F04FC00CF04EC00BF00CAE03D00B6C6C
:10566000E86A0C560CC022F00BC021F055C31BF0A9
:105670001C6A7FEC02F0606F14C061F061C014F02E
:1056800060C013F0020E33EC02F09C6F00EEDAF013
:105690009C51EBCF0BF00BC0D7F061C014F060C091
:1056A00013F0010E33EC02F09C6F00EEDAF09C5127
:1056B000EBCF0BF00BC0D8F061C014F060C013F05A
:1056C000000E33EC02F09C6F00EEDAF09C51EBCF51
:1056D0000BF00BC0D9F063BF05D0635307E1640E34
:1056E000625D04E2E4C00BF00BC0D4F0000163BFC4
:1056F00005D0635307E10A0E625D04E2E4C00BF0DB
:105700000BC0D5F0000161BF05D0615307E1640E05
:10571000605D04E2E4C00BF00BC0D7F0000161BF94
:1057200005D0615307E10A0E605D04E2E4C00BF0AE
:105730000BC0D8F0000144AA04D0F4C00BF00BC099
:10574000D4F081AC07D0D4510F6EFE0E0F140B6E47
:105750000BC0D4F081AA07D0D6510F6EFE0E0F14E5
:105760000B6E0BC0D6F081A807D0D7510F6EFE0E7E
:105770000F140B6E0BC0D7F081A607D0D9510F6E56
:10578000FE0E0F140B6E0BC0D9F083A007D0D551BD
:105790000F6EFE0E0F140B6E0BC0D5F083A207D058
:1057A000D8510F6EFE0E0F140B6E0BC0D8F09A512D
:1057B000E8A20DD0E4C00BF00BC0D4F0E4C00BF0B5
:1057C0000BC0D5F0E4C00BF00BC0D6F00ED043A058
:1057D0000CD0EAC00BF00BC0D4F0F1C00BF00BC042
:1057E000D5F0F1C00BF00BC0D6F042AE0CD0EAC041
:1057F0000BF00BC0D7F0F1C00BF00BC0D8F0F1C02C
:105800000BF00BC0D9F0840E026E020E086E840EEF
:10581000036E010E046E050E096ED451136EEFEC8B
:1058200001F0840E026E020E086E840E036E010EED
:10583000046E050E096ED551136EEFEC01F0840E67
:10584000026E020E086E840E036E010E046E050ECB
:10585000096ED651136EEFEC01F0840E026E020E4B
:10586000086E840E036E010E046E050E096ED7518C
:10587000136EEFEC01F0840E026E020E086E840EC1
:10588000036E010E046E050E096ED851136EEFEC17
:1058900001F0840E026E020E086E840E036E010E7D
:1058A000046E050E096ED951136EEFEC01F096945B
:1058B0008D8496948D941200449A9551E8AE01D04F
:1058C000448A95C00CF094C00BF00CAE03D00B6C66
:1058D000E86A0C560CC022F00BC021F055C31BF037
:1058E0001C6A7FEC02F0946F14C095F095C014F020
:1058F00094C013F0020E33EC02F09C6F00EEDAF06D
:105900009C51EBCF0BF00BC0D7F095C014F094C0B6
:1059100013F0010E33EC02F09C6F00EEDAF09C51B4
:10592000EBCF0BF00BC0D8F095C014F094C013F07F
:10593000000E33EC02F09C6F00EEDAF09C51EBCFDE
:105940000BF00BC0D9F044AA04D0F4C00BF00BC08C
:10595000D7F036EF41F093968A9693988A98939C65
:105960008A9C939A8A9A95968C9649C0BFF048C0B3
:10597000BEF047C0BDF046C0BCF0B76B010EB66FBD
:10598000B7530CE1330EB65D09E2010E18EC02F0DC
:10599000CBEC40F0B62B000EB723F2E382B23BD043
:1059A000010E42B4000E3B6E010E42B6000E3B16D5
:1059B00008E0000E42BC010E010AD8B4429CD8A4F3
:1059C000428C4290429242944296429E43900301FE
:1059D000516B526B00EEF6F0EF6A449C42BC828041
:1059E00042AC82900001BB6BBA6B82B214D0BA2B6E
:1059F000000EBB23030E146E200E26EC02F0050EE3
:105A0000BB5D06E303E1DD0EBA5D02E3000104D0F5
:105A1000CBEC40F0EAD712008290429C976B8392C5
:105A200083900EEC00F0800E016E19EC00F01D0E5C
:105A3000F76E440EF66E3BEC01F01D0EF76E5A0E3B
:105A4000F66E3BEC01F0F4C00BF00BC0D4F0F4C0E8
:105A50000BF00BC0D5F0F4C00BF00BC0D6F0F4C0C7
:105A60000BF00BC0D7F0F4C00BF00BC0D8F0F4C0B3
:105A70000BF00BC0D9F036EC41F082A2FED7030147
:105A8000140E546F4FC022F04EC021F055C31BF0CE
:105A90001C6A7FEC02F05A6E14C05BF05B5003018D
:105AA0005503F3CF5BF05A505503F3CF5AF0F4503F
:105AB0005B2655AF02D05A505B5E51C05DF050C0BE
:105AC0005CF068C06CF067C06BF06AC06EF069C0D3
:105AD0006DF070C076F06FC075F072C078F071C074
:105AE00077F000016F51735D796F705174597A6F5F
:105AF0009A51E8A606D0C451795D796FC5517A599B
:105B00007A6F43829AA1439243849AA34394438A2F
:105B10009AA5439A66C0B0F043869AA743964388F5
:105B20009AA94398438C9AAB439C448043AE4490DB
:105B300055C37DF059C37BF07C6B42889AAD429887
:105B4000428A9AAF429AB9C08BF0B8C08AF03DC37E
:105B500081F03CC380F03BC37FF03AC37EF041C389
:105B600085F040C384F03FC383F03EC382F043C35B
:105B700087F042C386F0458A9BA1459AB051030144
:105B80005503F4CFC9F0F3CFC8F086C389F085C3BD
:105B900088F0000182B41CD0140E18EC02F082B41C
:105BA00016D09607010E965D02E21A0E966F0F0E42
:105BB000965D0AE1010E43BC000E3B6E010E43B838
:105BC000000E3B1201E096070301140E546F000112
:105BD00082B61CD0140E18EC02F082B616D0962BAA
:105BE0001B0E965D02E3010E966F0F0E965D0AE1A5
:105BF000010E43BC000E3B6E010E43B8000E3B127B
:105C000001E0962B0301140E546F000180BC0AD0F2
:105C1000140E18EC02F080BC02D0FF0E976F030147
:105C2000140E546F000180BE0AD0140E18EC02F05E
:105C300080BE02D0010E976F0301140E546F000155
:105C4000010E82B2000E3B6E010E03015453D8A424
:105C5000000E3B120001D8B4B8D10E0E965D010EB5
:105C6000D8A4000E3B6E010E82B2000E3B1606E079
:105C7000439C0301140E546F0001A7D15BC047F091
:105C80005AC046F05DC049F05CC048F0000E66BFE7
:105C9000FF0E495C07E049506619D8B0800A800BB6
:105CA0001EE003D04850665D1AE248500001C45D12
:105CB000486E4950C559496EC4514626C5514722C0
:105CC000C651465CC75147584750C719D8B0800ADB
:105CD00006E7C651465C466EC7514758476E6CC0D2
:105CE00068F06BC067F06EC06AF06DC069F076C096
:105CF00070F075C06FF078C072F077C071F07551B8
:105D00007925736F76517A21746F9A51E8A604D081
:105D1000C4517327C55174239A8143A29A919A83DF
:105D200043A49A939A8543AA9A95B0C066F09A873D
:105D300043A69A979A8943A89A999A8B43AC9A9BBF
:105D4000438E44A0439E81C03DF380C03CF37FC09E
:105D50003BF37EC03AF385C041F384C040F383C077
:105D60003FF382C03EF387C043F386C042F38BC04B
:105D7000B9F08AC0B8F09B8145AA9B917DC055F3CC
:105D800003015551B40DF3CFC4F0F4CFC5F0555114
:105D9000680DF3CFC6F0F4CFC7F00001C7276651F6
:105DA00003015503F4CFC9F0F3CFC8F055510A0DE4
:105DB000F3CFCAF0F4CFCBF05551640DF3CFCCF054
:105DC000F4CFCDF07BC059F300019A8D42A89A9D83
:105DD0009A8F42AA9A9F89C086F388C085F366513C
:105DE00003015503F4CFC9F0F3CFC8F0AA6A040E3B
:105DF000A96E00016751D3EC01F06851D3EC01F0BA
:105E0000AA6A060EA96E6951D3EC01F06A51D3EC6F
:105E100001F0AA6A080EA96E6F51D3EC01F070511F
:105E2000D3EC01F0AA6A0A0EA96E7151D3EC01F00D
:105E30007251D3EC01F0AA6A0C0EA96E7351D3EC27
:105E400001F07451D3EC01F0AA6A0E0EA96E6651EE
:105E5000D3EC01F0AA6A0F0EA96E9A51D3EC01F0AF
:105E6000AA6A1E0EA96E9B51D3EC01F0AA6A100E0D
:105E7000A96E03015951D3EC01F0AA6A110EA96E63
:105E800003015551D3EC01F0AA6A120EA96E030169
:105E90003A51D3EC01F003013B51D3EC01F0030183
:105EA0003C51D3EC01F003013D51D3EC01F0AA6A5F
:105EB000160EA96E03013E51D3EC01F003013F51D0
:105EC000D3EC01F003014051D3EC01F00301415147
:105ED000D3EC01F0AA6A1A0EA96E03014251D3EC69
:105EE00001F003014351D3EC01F0AA6A1F0EA96E21
:105EF0000001B851D3EC01F0B951D3EC01F0AA6A1A
:105F00001C0EA96E86C314F085C313F0186A0A0E1E
:105F1000176E68EC02F0266E14C027F02650D3EC02
:105F200001F02750D3EC01F0166A070E156EA10E92
:105F3000146E200E136E85C31BF086C31CF01D6A01
:105F40001E6A3DEC02F014C084F313C083F3FFEC2F
:105F500043F0800E016E10EC00F020EC27F082A2DE
:105F6000FED7000E42B0010E3B6E000E42B2010E93
:105F70003B1202E095968C869A51E8A616D0C45141
:105F800046245E6EC55147205F6E5E50C65D5F5011
:105F9000C7595F50C719D8B0800A06E6C6515E5C83
:105FA0005E6EC7515F585F6E04D047C05FF046C059
:105FB0005EF047C09AF346C099F3C9EC44F09CC325
:105FC0005FF09BC35EF0429C1200010E965DD8A468
:105FD00050D0975103015503F3CF26F0F4CF27F0AB
:105FE00055AF01D0275E000197AF03D00301555193
:105FF000275E26505A2627505B220001975301E066
:1060000042805A50C65D5B50C7595B50C719D8B023
:10601000800A06E6C6515A5C5A6EC7515B585B6EE1
:106020005BAE04D0C6515A26C7515B22800E016E6A
:1060300019EC00F01D0EF76E700EF66E3BEC01F0E1
:10604000800E016E030E076E5BC022F05AC021F075
:1060500055C31BF01C6A7FEC02F01B6E14C01CF0D1
:106060006FEC00F0050E43EC01F09CEC43F038EFD0
:1060700037F0020E965DD8A450D097510301550316
:10608000F3CF26F0F4CF27F055AF01D0275E000103
:1060900097AF03D003015551275E26505C26275049
:1060A0005D220001975301E042825C50C85D5D5063
:1060B000C9595D50C919D8B0800A07E6B05103012B
:1060C0005503F4CF5DF0F3CF5CF000015DAE02D07C
:1060D0005D6A5C6A800E016E19EC00F01D0EF76EB1
:1060E000820EF66E3BEC01F0800E016E030E076E21
:1060F0005DC022F05CC021F055C31BF01C6A7FEC30
:1061000002F01B6E14C01CF06FEC00F0050E43ECA7
:1061100001F09CEC43F038EF37F0030E965DD8A405
:106120004AD0975103015503F3CF26F0F4CF27F05F
:1061300055AF01D0275E000197AF03D00301555141
:10614000275E265000016B2727506C236B51C65DDC
:106150006C51C7596C51C719D8B0800A04E6C7C042
:106160006CF0C6C06BF06C51E8AE02D06C6B6B6B20
:10617000800E016E19EC00F01D0EF76E940EF66E97
:106180003BEC01F0800E016E030E076E6CC022F036
:106190006BC021F055C31BF01C6A7FEC02F01B6E34
:1061A00014C01CF06FEC00F0050E43EC01F09CEC09
:1061B00043F038EF37F0040E965DD8A44ED09751D7
:1061C00003015503F3CF26F0F4CF27F055AF01D0EC
:1061D000275E000197AF03D003015551275E26507B
:1061E00000016D2727506E236D51C85D6E51C9594E
:1061F0006E51C919D8B0800A07E6B05103015503A2
:10620000F4CF6EF0F3CF6DF000016E51E8AE02D026
:106210006E6B6D6B800E016E19EC00F01D0EF76E4B
:10622000A60EF66E3BEC01F0800E016E030E076EBB
:106230006EC022F06DC021F055C31BF01C6A7FECCC
:1062400002F01B6E14C01CF06FEC00F0050E43EC66
:1062500001F09CEC43F038EF37F0050E965DD8A4C2
:106260004AD0975103015503F3CF26F0F4CF27F01E
:1062700055AF01D0275E000197AF03D00301555100
:10628000275E265000017527275076237551CE5D75
:106290007651CF597651CF19D8B0800A04E6CFC0D5
:1062A00076F0CEC075F07651E8AE02D0766B756BA5
:1062B000800E016E19EC00F01D0EF76EB80EF66E32
:1062C0003BEC01F0800E016E030E076E76C022F0EB
:1062D00075C021F055C31BF01C6A7FEC02F01B6EE9
:1062E00014C01CF06AEC00F0050E43EC01F09CECCD
:1062F00043F038EF37F0060E965DD8A44AD0975198
:1063000003015503F3CF26F0F4CF27F055AF01D0AA
:10631000275E000197AF03D003015551275E265039
:1063200000017727275078237751D05D7851D159D4
:106330007851D119D8B0800A04E6D1C078F0D0C025
:1063400077F07851E8AE02D0786B776B800E016EF3
:1063500019EC00F01D0EF76ECA0EF66E3BEC01F064
:10636000800E016E030E076E78C022F077C021F018
:1063700055C31BF01C6A7FEC02F01B6E14C01CF0AE
:106380006AEC00F0050E43EC01F09CEC43F038EFB2
:1063900037F0070E965DD8A4AFD09751030155038F
:1063A000F3CF26F0F4CF27F055AF01D0275E0001E0
:1063B00097AF03D003015551275E2650000179277E
:1063C00027507A239A51E8B63FD0C651795DC7511C
:1063D0007A597A51C719D8B0800A04E6C7C07AF052
:1063E000C6C079F003015551A40DF3CF0BF0F4CFE3
:1063F0000CF00D6A0E6A5551010DF3500C26F45045
:106400000D22000E0E2279C013F07AC014F0000E97
:1064100014BEFF0E156E166E13500B5C14500C5804
:1064200015500D5816500E580E501618D8B0800A38
:10643000000109E603015551A40DF3CF79F0F4CF23
:106440007AF000017A2735D0C451795DC5517A5967
:106450007A51C519D8B0800A04E6C5C07AF0C4C024
:1064600079F003015551F00DF3CF0BF0F4CF0CF0A0
:106470000D6A0E6A79C013F07AC014F0000E14BED3
:10648000FF0E156E166E13500B5C14500C58155001
:106490000D5816500E580E501618D8B0800A00012C
:1064A00007E603015551F00DF3CF79F0F4CF7AF000
:1064B0000001800E016E19EC00F01D0EF76EDC0E6F
:1064C000F66E3BEC01F0800E016E030E076E7AC093
:1064D00022F079C021F055C31BF01C6A7FEC02F05A
:1064E0001B6E14C01CF06FEC00F0050E43EC01F0C5
:1064F0009CEC43F038EF37F0080E965D23E197519E
:106500007B257B6F000E97BFFF0E7C217C6F800E7A
:10651000016E19EC00F01D0EF76EEE0EF66E3BEC00
:1065200001F0800E016E030E076E7CC01CF07BC074
:106530001BF06FEC00F0050E43EC01F09CEC43F017
:1065400038EF37F0090E965DD8A452D09751E8BEC7
:1065500003D0975301E0458A9751E8AE01D0459AA0
:10656000800E016E19EC00F01E0EF76E000EF66E36
:106570003BEC01F045AA0AD04C0E43EC01F0430E6F
:1065800043EC01F0440E43EC01F009D04C0E43EC17
:1065900001F0450E43EC01F0440E43EC01F0800E97
:1065A000016EC00E19EC00F0200E43EC01F0000E5D
:1065B00043EC01F0200E43EC01F04D0E43EC01F0F2
:1065C000200E43EC01F0010E43EC01F0200E43ECF1
:1065D00001F043EC01F043EC01F0040E43EC01F058
:1065E0001E0EF76E120EF66E3BEC01F038EF37F030
:1065F0000A0E965D2CE19751E8BE03D0975301E057
:1066000043949751E8AE01D04384800E016E19EC9B
:1066100000F01E0EF76E1E0EF66E3BEC01F043A46A
:1066200009D04F0E43EC01F0460E43EC01F043EC71
:1066300001F009D0200E43EC01F04F0E43EC01F0C5
:106640004E0E43EC01F0D8EC43F038EF37F00B0E70
:10665000965D46E19751E8BE03D0975301E0438A27
:106660009751E8AE01D0439A800E016E19EC00F00C
:106670001E0EF76E300EF66E3BEC01F043AA04D00E
:10668000420E43EC01F003D0410E43EC01F0800ECA
:10669000016EC00E19EC00F0200E43EC01F0000E6C
:1066A00043EC01F0200E43EC01F04D0E43EC01F001
:1066B000200E43EC01F0010E43EC01F0200E43EC00
:1066C00001F043EC01F043EC01F0040E43EC01F067
:1066D0001E0EF76E440EF66E3BEC01F038EF37F00D
:1066E0000C0E965DD8A451D09751E8BE04D09753B4
:1066F00002E0B40EB06F9751E8AE02D05A0EB06F00
:10670000B05103015503F4CFC9F0F3CFC8F0800EA8
:10671000016E19EC00F01E0EF76E500EF66E3BEC9B
:1067200001F0800E016E030E076E0001B0516DEC9A
:1067300000F0050E43EC01F0800E016EC00E19EC66
:1067400000F0200E43EC01F0000E43EC01F0200EAF
:1067500043EC01F04D0E43EC01F0200E43EC01F050
:10676000010E43EC01F0200E43EC01F043EC01F08C
:1067700043EC01F0040E43EC01F01E0EF76E620EC6
:10678000F66E3BEC01F038EF37F00D0E965D4CE104
:106790009751E8BE03D0975301E043869751E8AE86
:1067A00001D04396800E016E19EC00F01E0EF76EBC
:1067B0006E0EF66E3BEC01F043B607D01E0EF76E80
:1067C0007E0EF66E3BEC01F006D01E0EF76E860EC6
:1067D000F66E3BEC01F0800E016EC00E19EC00F07D
:1067E000200E43EC01F0000E43EC01F0200E43ECD0
:1067F00001F04D0E43EC01F0200E43EC01F0010ED0
:1068000043EC01F0200E43EC01F043EC01F043ECCB
:1068100001F0040E43EC01F01E0EF76E8E0EF66EC4
:106820003BEC01F038EF37F00E0E965DD8A44DD05A
:106830009751E8BE04D0975302E04388438C9751A8
:10684000E8AE02D04398438C800E016E19EC00F044
:106850001E0EF76E9A0EF66E3BEC01F043BC07D0AD
:106860001E0EF76EA40EF66E3BEC01F00FD043B88F
:1068700007D01E0EF76EB00EF66E3BEC01F006D0A0
:106880001E0EF76EBC0EF66E3BEC01F0800E016E34
:10689000C00E19EC00F0200E43EC01F0000E43ECAA
:1068A00001F0200E43EC01F04D0E43EC01F0200E00
:1068B00043EC01F0010E43EC01F01E0EF76EC80E22
:1068C000F66E3BEC01F038EF37F00F0E965DD8A472
:1068D00051D09751E8AE11D0030E895D0AE303E170
:1068E000E90E885D06E30A0E0001885F000E895BF1
:1068F00004D0030E896FE80E886F9751E8BE11D05F
:1069000097530FE0270E895D100E01E1885D05E2C7
:106910000A0E8827000E892304D0270E896F100ED7
:10692000886F800E016E19EC00F01E0EF76ED80E07
:10693000F66E3BEC01F0270E895D100E01E1885DDB
:1069400003E2200E43EC01F0800E016E076A89C05D
:106950001CF088C01BF06FEC00F0200E43EC01F03F
:10696000480E43EC01F07A0E43EC01F09CEC43F04E
:1069700038EF37F0100E965D2EE1800E016E19ECA7
:1069800000F01E0EF76EE60EF66E3BEC01F08EC3C5
:1069900029F08DC328F08CC327F08BC326F0010E9D
:1069A000A7EC00F0200E43EC01F043EC01F043ECC7
:1069B00001F043EC01F043EC01F0800E016EC00EDB
:1069C00019EC00F0160E066E020E1C6E120E2BEC69
:1069D00001F038EF37F0110E965DD8A45BD09751D7
:1069E000E8BE11D097530FE0040E7D5D02E1020E68
:1069F0007D6F0A0E7D5D02E1040E7D6F140E7D5DDC
:106A000002E10A0E7D6F9751E8AE0FD00A0E7D5D50
:106A100002E1140E7D6F040E7D5D02E10A0E7D6FB2
:106A2000020E7D5D02E1040E7D6F800E016E19EC99
:106A300000F01E0EF76EF40EF66E3BEC01F0140E35
:106A40007D5D07E11F0EF76E000EF66E3BEC01F068
:106A50001AD00A0E7D5D07E11F0EF76E0A0EF66E64
:106A60003BEC01F010D0040E7D5D07E11F0EF76EC8
:106A7000140EF66E3BEC01F006D01F0EF76E1E0EE4
:106A8000F66E3BEC01F09CEC43F00301110E5C6FE1
:106A90000001EED1120E965D29E10301010EA06FF7
:106AA00081C0A4F380C0A3F37FC0A2F37EC0A1F392
:106AB0000001F6EC45F0A8C381F0A7C380F0A6C39F
:106AC0007FF0A5C37EF00301140E546F110E5C5DC0
:106AD000000103E1130E966F02D0110E966F0301B1
:106AE000120E5C6F0001C9EF2DF0C2D1130E965D3E
:106AF00029E10301020EA06F85C0A4F384C0A3F3B3
:106B000083C0A2F382C0A1F30001F6EC45F0A8C354
:106B100085F0A7C384F0A6C383F0A5C382F0030168
:106B2000140E546F120E5C5D000103E1140E966F9B
:106B300002D0120E966F0301130E5C6F0001C9EFB5
:106B40002DF096D1140E965D31E197518625866F12
:106B5000000E97BFFF0E8721876F8751E8AE02D0E6
:106B6000876B866B800E016E19EC00F01F0EF76EBE
:106B7000280EF66E3BEC01F0800E016E040E076EDF
:106B800087C01CF086C01BF06FEC00F0200E43ECB9
:106B900001F06D0E43EC01F0200E43EC01F09CEC93
:106BA00043F00301140E5C6F000162D1150E965D77
:106BB0002BE19751E8AE01D042989751E8BE03D03F
:106BC000975301E04288800E016E19EC00F01F0E11
:106BD000F76E360EF66E3BEC01F042B809D04F0E60
:106BE00043EC01F0460E43EC01F043EC01F009D018
:106BF000200E43EC01F04F0E43EC01F04E0E43EC3F
:106C000001F0D8EC43F034D1160E965D2BE197518C
:106C1000E8AE01D0429A9751E8BE03D0975301E005
:106C2000428A800E016E19EC00F01F0EF76E480EBE
:106C3000F66E3BEC01F042BA09D04F0E43EC01F086
:106C4000460E43EC01F043EC01F009D0200E43EC7A
:106C500001F04F0E43EC01F04E0E43EC01F0D8EC86
:106C600043F006D1170E965DD8A468D09751E8AED0
:106C700020D08B51250A800ED8B48A1904E1120E57
:106C80008B6FC00E8A6F8B514B0A8A1104E1250E5F
:106C90008B6F800E8A6F8B51960A8A1103E14B0E1F
:106CA0008B6F8A6B8B51E10A8A1103E1960E8B6F11
:106CB0008A6B9751E8BE23D0975321E08B51960AF7
:106CC0008A1103E1E10E8B6F8A6B8B514B0A8A119B
:106CD00003E1960E8B6F8A6B8B51250A800ED8B418
:106CE0008A1903E14B0E8B6F8A6B8B51120AC00E0F
:106CF000D8B48A1904E1250E8B6F800E8A6F800E3E
:106D0000016E19EC00F01F0EF76E5A0EF66E3BEC9A
:106D100001F0270E8B5D100E01E18A5D03E2200E6B
:106D200043EC01F0800E016E076A8BC01CF08AC034
:106D30001BF06FEC00F09CEC43F09AD0180E965DBF
:106D40002BE19751E8BE03D0975301E0438297515E
:106D5000E8AE01D04392800E016E19EC00F01F0ED8
:106D6000F76E6A0EF66E3BEC01F043A20AD0200EDD
:106D700043EC01F04F0E43EC01F04E0E43EC01F0FA
:106D800008D04F0E43EC01F0460E43EC01F043EC0B
:106D900001F0D8EC43F06CD0190E965D2BE19751C1
:106DA000E8AE01D044909751E8BE03D0975301E07C
:106DB0004480800E016E19EC00F01F0EF76E7C0E01
:106DC000F66E3BEC01F044B009D04F0E43EC01F0FD
:106DD000460E43EC01F043EC01F009D0200E43ECE9
:106DE00001F04F0E43EC01F04E0E43EC01F0D8ECF5
:106DF00043F03ED01A0E965D3BE19751E8AE01D0CC
:106E00008ED89751E8BE03D0975301E030D9800E59
:106E1000016E19EC00F01F0EF76E8E0EF66E3BEC55
:106E200001F0800E016EC00E19EC00F0200E43EC54
:106E300001F0000E43EC01F0200E43EC01F04D0E8A
:106E400043EC01F0200E43EC01F0010E43EC01F0A5
:106E5000200E43EC01F043EC01F043EC01F0040E92
:106E600043EC01F01F0EF76EA40EF66E3BEC01F042
:106E7000976B010E82B4000E3B6E010E82B6000EBF
:106E80003B1203E0CBEC40F0F4D7BB6BBA6B010EC6
:106E900080BC000E3B6E010E80BE000E3B1211E066
:106EA000030156510001BA27000EBB23BA51985D69
:106EB000BB51995906E3010E18EC02F0CBEC40F0FF
:106EC000E6D7995303E1330E985D05E3190E0001EF
:106ED000985F000E995B000E80BC010E3B6E000EA9
:106EE00080BE010E3B16000E82B6010E3B16000E50
:106EF00082B4010E3B16000E82B2010E3B160BE06F
:106F0000010E996FF40E986FCBEC40F003015453CF
:106F1000000101E0E0D7C9EF2DF0429C1200448E41
:106F2000800E016E19EC00F01F0EF76EB00EF66EBB
:106F30003BEC01F0800E016EC00E19EC00F01F0E4C
:106F4000F76EC60EF66E3BEC01F082A6FED7936B91
:106F5000926B4590458293988A88070E935DD00E78
:106F600001E1925D34E24B50C15D07E14A50C05DE2
:106F700004E1922B000E932306D04BC0C1F04AC00F
:106F8000C0F0936B926B800E016EC00E19EC00F096
:106F9000030E076E4BC022F04AC021F055C31BF010
:106FA0001C6A7FEC02F01B6E14C01CF06AEC00F04F
:106FB000CBEC40F082B20AD093988A98449E0301A9
:106FC000516B429E140E546F00011200C6D7939865
:106FD0008A984B6A4A6A800E016EC00E19EC00F066
:106FE0001F0EF76ED00EF66E3BEC01F0449E4592FC
:106FF000458093968A866F514A5C0B6E70514B5850
:107000000C6E0CAE2CD06F514A5C266E70514B58F2
:10701000276E27C022F026C021F055C31BF01C6A42
:107020007FEC02F08C6F14C08DF0800E016EC00EEC
:1070300019EC00F0030E076E8DC01CF08CC01BF025
:107040006AEC00F0CBEC40F0010E82B2000E3B6E19
:10705000000E42BE010E3B1201E001D0CCD7939648
:107060008A960301516B140E546F00011200448E76
:10707000800E016E19EC00F01F0EF76EB00EF66E6A
:107080003BEC01F0800E016EC00E19EC00F01F0EFB
:10709000F76EC60EF66E3BEC01F082A4FED7936B42
:1070A000926B4DC0C3F04CC0C2F045944586939C92
:1070B0008A8C070E935DD00E01E1925D32E24D5055
:1070C000C35D07E14C50C25D04E1922B000E932397
:1070D00006D04DC0C3F04CC0C2F0936B926B800ED3
:1070E000016EC00E19EC00F0030E076E4DC022F0C9
:1070F0004CC021F055C31BF01C6A7FEC02F01B6EE4
:1071000014C01CF06AEC00F0CBEC40F082B208D066
:10711000449E0301526B4390140E546F0001120001
:10712000C8D7939C8A9C4D6A4C6A800E016EC00E33
:1071300019EC00F01F0EF76ED00EF66E3BEC01F06E
:10714000449E45964584939A8A8A71514C5C0B6E95
:1071500072514D580C6E0CAE2CD071514C5C266E99
:1071600072514D58276E27C022F026C021F055C31A
:107170001BF01C6A7FEC02F08C6F14C08DF0800E47
:10718000016EC00E19EC00F0030E076E8DC01CF0EE
:107190008CC01BF06AEC00F0CBEC40F0010E82B228
:1071A000000E3B6E000E43B0010E3B1201E001D019
:1071B000CCD7939A8A9A0301526B140E546F000134
:1071C000120002EE28F0E9CFDEFFEACFDEFF030176
:1071D0009F6B0001B9EC45F01FEEE9F01DEC03F0E8
:1071E00013EEC4F0500EE75204E0E6CFEEFFE82EB7
:1071F000FAD7EF6A01EEB1F012EE28F0030E3EEC82
:1072000003F0EF6A1F0EF76ED80EF66E01EEB1F0C6
:107210005CEC03F03B6E000E42B0010E3B12000E20
:1072200042B2010E3B1204E000EEF6F0EF6A1200EB
:10723000010EA56FA26B00EEF6F0A551EB500B6EA0
:107240002A0E0B5C08E000EEF6F0A551EB500B6E39
:10725000A21BA52BF0D7A52B00EEF6F0A551EB5005
:10726000186E0C0EF66E200EF76EF86A1768172A65
:1072700017500F0806E30900F550185CF8E117C035
:10728000A3F0A339F00BA46FA52B00EEF6F0A551E7
:10729000EB50186E1C0EF66E200EF76EF86A17682B
:1072A000172A17500F0806E30900F550185CF8E19B
:1072B00017C0A3F0A451A327A251A35D01E01200BF
:1072C00002EE28F0E9CFDEFFEACFDEFF0301020E77
:1072D0009F6F0001B9EC45F01FEEE9F01DEC03F0E3
:1072E00013EEC4F0500EE75204E0E6CFEEFFE82EB6
:1072F000FAD7EF6A02012C510B6E2E0E0B5C0001C7
:1073000001E0120001EEB1F012EE28F0020EE6CF1D
:10731000EEFFE82EFCD7EF6A01EEB1F020EC00F0B2
:107320000301236F01EEB1F012EE28F0030EF36EAD
:10733000020E35EC03F0EF6A01EEB1F020EC00F044
:107340001EC035F01DC034F01CC033F01BC032F03D
:107350001AEC09F035C027F334C026F333C025F307
:1073600032C024F3010E03012353D8A4000E3B6E58
:10737000356A346A336A326A27C339F026C338F073
:1073800025C337F024C336F0B2EC06F03B160001FB
:1073900001E0458CB40E0301235D010ED8A4000E5C
:1073A0003B6E356A346A336A326A27C339F026C3C2
:1073B00038F025C337F024C336F0B2EC06F03B16A4
:1073C000000101E0458C01EEB1F012EE28F0060E4E
:1073D000F36E020E35EC03F0EF6A01EEB1F020EC33
:1073E00000F01EC035F01DC034F01CC033F01BC0CF
:1073F00032F01AEC09F035C06CF334C06BF333C0D3
:107400006AF332C069F3396A386A480E376E850EFE
:10741000366E6CC335F06BC334F06AC333F069C3A6
:1074200032F009EC08F035C029F034C028F033C040
:1074300027F032C026F027C339F026C338F025C321
:1074400037F024C336F029C035F028C034F027C007
:1074500033F026C032F07BEC07F035C027F334C0A0
:1074600026F333C025F332C024F3396A386A700E2C
:10747000376E840E366E27C335F026C334F025C32D
:1074800033F024C332F009EC08F035C029F034C0E1
:1074900028F033C027F032C026F00301235116EC48
:1074A00009F029C039F028C038F027C037F026C0CD
:1074B00036F07BEC07F035C02BF334C02AF333C031
:1074C00029F332C028F3356A346A340E336E850EE0
:1074D000326E2BC339F02AC338F029C337F028C3E2
:1074E00036F0F7EC06F00108000101E0120002EEB0
:1074F00028F0E9CFDEFFEACFDEFF0301030E9F6F26
:107500000001B9EC45F01FEEE9F01DEC03F013EEBD
:10751000C4F0500EE75204E0E6CFEEFFE82EFAD7B3
:10752000EF6A02EE28F0EECFF3FFEFCFF4FFF35057
:10753000530AF41002E10301297F000102EE28F052
:10754000E9CFDEFFEACFDEFF0301040E9F6F0001EB
:10755000B9EC45F01FEEE9F01DEC03F013EEC4F0BA
:10756000500EE75204E0E6CFEEFFE82EFAD7EF6ABE
:1075700002012D510B6E2E0E0B5C000101E012007A
:1075800001EEB1F012EE28F0030EE6CFEEFFE82E8A
:10759000FCD7EF6A01EEB1F020EC00F00301236F9D
:1075A00001EEB1F012EE28F0040EF36E020E35EC8F
:1075B00003F0EF6A01EEB1F020EC00F01EC035F0F0
:1075C0001DC034F01CC033F01BC032F01AEC09F0BF
:1075D00035C027F334C026F333C025F332C024F37B
:1075E000010E03012353D8A4000E3B6E356A346AA2
:1075F000336A326A27C339F026C338F025C337F01F
:1076000024C336F0B2EC06F03B16000E45BC010E6A
:107610003B16000104E000EEF6F0EF6A120001EE06
:10762000B1F012EE28F0070EF36E020E35EC03F007
:10763000EF6A01EEB1F020EC00F01EC035F01DC085
:1076400034F01CC033F01BC032F01AEC09F035C026
:107650006CF334C06BF333C06AF332C069F3396A38
:10766000386A480E376E850E366E6CC335F06BC3C4
:1076700034F06AC333F069C332F009EC08F035C066
:1076800029F034C028F033C027F032C026F027C3D9
:1076900039F026C338F025C337F024C336F029C0AB
:1076A00035F028C034F027C033F026C032F07BEC30
:1076B00007F035C027F334C026F333C025F332C0BA
:1076C00024F3396A386A700E376E840E366E27C31B
:1076D00035F026C334F025C333F024C332F009EC6F
:1076E00008F035C029F034C028F033C027F032C08C
:1076F00026F00301235116EC09F029C039F028C007
:1077000038F027C037F026C036F07BEC07F035C0E4
:107710002FF334C02EF333C02DF332C02CF3356A6F
:10772000346A340E336E860E326E2FC339F02EC398
:1077300038F02DC337F02CC336F0BFEC06F001084B
:10774000000101E0120002EE28F0E9CFDEFFEACFEF
:10775000DEFF0301050E9F6F0001B9EC45F01FEE3F
:10776000E9F01DEC03F013EEC4F0500EE75204E014
:10777000E6CFEEFFE82EFAD7EF6A02EE28F0EECF62
:10778000F3FFEFCFF4FFF350570AF41002E10301C7
:107790002D7F000102EE28F0E9CFDEFFEACFDEFF09
:1077A0000301090E9F6F0001B9EC45F01FEEE9F0EF
:1077B0001DEC03F013EEC4F0500EE75204E0E6CFE8
:1077C000EEFFE82EFAD7EF6A02EE28F020EC00F088
:1077D0000301386F1CC039F301EEB1F012EE28F04E
:1077E000010E3EEC03F0EF6A0101B1510B6E350E54
:1077F0000B5C000104E30301382B000E39239C0EBF
:107800000301395D000108E305E1410E0301385D24
:10781000000102E300011200D00E356E0F0E346E2F
:10782000490E336E800E326E2BC339F02AC338F006
:1078300029C337F028C336F06FEC08F035C029F0C3
:1078400034C028F033C027F032C026F0396A386AD5
:10785000340E376E860E366E29C035F028C034F0EF
:1078600027C033F026C032F009EC08F035C06CF3C5
:1078700034C06BF333C06AF332C069F36CC335F0C4
:107880006BC334F06AC333F069C332F098EC04F090
:1078900035C0AFF034C0AEF033C0ADF032C0ACF0A4
:1078A0002FC329F02EC328F02DC327F02CC326F0B8
:1078B00029C035F028C034F027C033F026C032F09C
:1078C00041C339F040C338F03FC337F03EC336F010
:1078D00079EC07F035C029F034C028F033C027F028
:1078E00032C026F029C039F028C038F027C037F060
:1078F00026C036F0AFC035F0AEC034F0ADC033F0C6
:10790000ACC032F06FEC08F035C029F034C028F07C
:1079100033C027F032C026F09A0E356E990E346EC1
:107920005E0E336E850E326E29C039F028C038F0F5
:1079300027C037F026C036F06FEC08F035C04BF3A7
:1079400034C04AF333C049F332C048F32BC335F097
:107950002AC334F029C333F028C332F03DC339F0D1
:107960003CC338F03BC337F03AC336F079EC07F04C
:1079700035C029F034C028F033C027F032C026F0DB
:107980009A0E356E990E346E5E0E336E850E326E23
:1079900029C039F028C038F027C037F026C036F0AB
:1079A0006FEC08F035C047F334C046F333C045F3FD
:1079B00032C044F347C339F046C338F045C337F00B
:1079C00044C336F047C335F046C334F045C333F003
:1079D00044C332F06FEC08F0BDEC08F003016D6FAA
:1079E00033C06EF334C06FF335C070F34BC339F05E
:1079F0004AC338F049C337F048C336F04BC335F0BB
:107A00004AC334F049C333F048C332F06FEC08F096
:107A1000BDEC08F00301716F33C072F334C073F32F
:107A200035C074F371516D255D6F72516E215E6FBB
:107A300073516F215F6F74517021606F60C335F0B7
:107A40005FC334F05EC333F05DC332F01CEC09F069
:107A500007EC06F035C080F334C07FF333C07EF30B
:107A600032C07DF3396A386A7A0E376E880E366E08
:107A700043C333F042C332F010EC09F009EC08F0D4
:107A800035C029F034C028F033C027F032C026F0CA
:107A9000356A500E346E470E336E8B0E326E29C02F
:107AA00039F028C038F027C037F026C036F07BEC1C
:107AB00007F035C07CF334C07BF333C07AF332C0B7
:107AC00079F37CC339F07BC338F07AC337F079C3DC
:107AD00036F07CC335F07BC334F07AC333F079C31E
:107AE00032F06FEC08F0BDEC08F003016D6F33C0AD
:107AF0006EF334C06FF335C070F380C339F07FC3C9
:107B000038F07EC337F07DC336F080C335F07FC3D5
:107B100034F07EC333F07DC332F06FEC08F0BDEC7F
:107B200008F00301716F33C072F334C073F335C0D2
:107B300074F371516D255D6F72516E215E6F7351DB
:107B40006F215F6F74517021606F60C335F05FC348
:107B500034F05EC333F05DC332F01CEC09F007EC87
:107B600006F035C0AFF034C0AEF033C0ADF032C077
:107B7000ACF0AFC029F0AEC028F0ADC027F0ACC06B
:107B800026F029C035F028C034F027C033F026C0D5
:107B900032F07CC339F07BC338F07AC337F079C355
:107BA00036F079EC07F035C029F034C028F033C046
:107BB00027F032C026F0356A346A7A0E336E880EAA
:107BC000326E29C039F028C038F027C037F026C0FF
:107BD00036F06FEC08F035C029F034C028F033C01F
:107BE00027F032C026F043C333F042C332F010EC2A
:107BF00009F029C039F028C038F027C037F026C076
:107C000036F07BEC07F0BDEC08F003016D6F33C07C
:107C10006EF334C06FF335C070F370530001D8A415
:107C20009FD003016F530001D8A49AD003016E5175
:107C3000395D0001D8A094D006E1030138516D5D93
:107C40000001D8B08DD003016D51385D716F6E5158
:107C50003959726F000E6F55736F000E7055746F47
:107C600080C339F07FC338F07EC337F07DC336F070
:107C700074C335F073C334F072C333F071C332F0A0
:107C80001AEC09F009EC08F035C029F034C028F0EE
:107C900033C027F032C026F0396A386A7A0E376E60
:107CA000880E366E29C035F028C034F027C033F076
:107CB00026C032F009EC08F035C0AFF034C0AEF0A9
:107CC00033C0ADF032C0ACF0AFC035F0AEC034F070
:107CD000ADC033F0ACC032F066EC03F035C06CF3ED
:107CE00034C06BF333C06AF332C069F36CC337F34B
:107CF0006BC336F36AC335F369C334F3356A346A48
:107D0000340E336E860E326E6CC339F06BC338F0AE
:107D10006AC337F069C336F06FEC08F035C029F05C
:107D200034C028F033C027F032C026F0D00E396EB0
:107D30000F0E386E490E376E800E366E29C035F044
:107D400028C034F027C033F026C032F009EC08F028
:107D50006FEC07F00301816F33C082F3000103D0A1
:107D60000301826B816B0301825304E15B0E815D31
:107D7000000104E3496A486A0001120003015551F9
:107D80008103F3CF48F0F4CF49F08203F350492642
:107D9000000149AE03D0496A486A120049C033F075
:107DA00048C032F010EC09F035C037F334C036F378
:107DB00033C035F332C034F34850BE5D136E4950C2
:107DC000BF59146E0AEC03F00B6E14C00CF00301E3
:107DD0005551050DF3CF0FF0F4CF10F0116A126A70
:107DE0001252000114E1115212E110500C5C0FE329
:107DF00003E10B500F5C0BE20001A82B030EA85D02
:107E000005E349C0BFF048C0BEF0A86B01D0A86B25
:107E10004BC335F04AC334F049C333F048C332F0A2
:107E200047C339F046C338F045C337F044C336F092
:107E300009EC08F035C0AFF034C0AEF033C0ADF09F
:107E400032C0ACF0AFC035F0AEC034F0ADC033F0EE
:107E5000ACC032F066EC03F035C06CF334C06BF3A9
:107E600033C06AF332C069F3356A346A340E336E54
:107E7000860E326E6CC339F06BC338F06AC337F0CC
:107E800069C336F06FEC08F035C029F034C028F033
:107E900033C027F032C026F0D00E396E0F0E386E88
:107EA000490E376E800E366E29C035F028C034F08A
:107EB00027C033F026C032F009EC08F035C06CF36F
:107EC00034C06BF333C06AF332C069F36CC333F36D
:107ED0006BC332F36AC331F369C330F36CC335F05B
:107EE0006BC334F06AC333F069C332F06FEC07F050
:107EF0000301816F33C082F347C335F046C334F0CA
:107F000045C333F044C332F0396A386A376A366A97
:107F1000F7EC06F03B6E4BC335F04AC334F049C36F
:107F200033F048C332F0396A386A376A366A33EC5C
:107F300007F03B1600011DE0680E03018127010ECA
:107F40008223356A346A340E336E870E326E33C341
:107F500039F032C338F031C337F030C336F07BEC40
:107F600007F035C033F334C032F333C031F332C0DD
:107F700030F3030145510001E8AE1DD0B40E0301FA
:107F80008127000E8223356A346A340E336E860EE2
:107F9000326E33C339F032C338F031C337F030C3F7
:107FA00036F07BEC07F035C033F334C032F333C026
:107FB00031F332C030F3000182C347F081C346F091
:107FC000030181510001BC5D136E03018251000168
:107FD000BD59146E0AEC03F00B6E14C00CF00C5279
:107FE00003E1060E0B5C0BE30001A72B030EA75D5C
:107FF00005E382C3BDF081C3BCF0A76B01D0A76BC2
:1080000000EEF6F0EF6AA75302E1000E01D0010E78
:108010003B6EA85302E1000E01D0010E3B1201E0BD
:10802000120082C3BDF081C3BCF049C0BFF048C09C
:10803000BEF01E0E03015B5D000101E212000301B0
:1080400055518103F3CF46F0F4CF47F08203F3504C
:10805000472647C09AF346C099F30001C9EC44F0A3
:108060009CC35FF09BC35EF043BE43D06F514A5C3C
:108070000B6E70514B580C6E70BFFF0E000E0D6AE8
:108080004BBE0D6870BFFF0E0D5A0E6A0DBE0E6816
:108090000B505E180BE10C505F1808E10D505FBEED
:1080A0000D2804E10E505FBE0E2801E04280000161
:1080B00071514C5C0B6E72514D580C6E72BFFF0EBD
:1080C000000E0D6A4DBE0D6872BFFF0E0D5A0E6A8E
:1080D0000DBE0E680B5048180BE10C50491808E112
:1080E0000D5049BE0D2804E10E5049BE0E2801E096
:1080F000428203015B6B000E42B0010E3B6E000E2C
:1081000042B2010E3B12000101E001D812009A5167
:10811000E8BA01D01200000E81B6010E3B6E000ECF
:1081200081B8010E3B12000E81BA010E3B12000E07
:1081300081BC010E3B1201E012009A51E8A824D044
:10814000610E146EA80E136E84C318F083C317F06B
:1081500068EC02F00A6EA06BA0510A5C13E3939ED8
:108160008A8E84C314F00301835126EC02F0939E9F
:108170008A9E84C314F00301835126EC02F00001AF
:10818000A02BEAE3938E06D0939E8A8E320E18ECD3
:1081900002F0938E1200E86A44B2010F83BC01081A
:1081A000D8A4010E3B6EE86A44B4010F83BE0108F7
:1081B000D8A4010E3B12D8B458D0020E18EC02F02D
:1081C000E86A44B2010F83BC0108D8A4010E3B6EDB
:1081D000E86A44B4010F83BE0108D8A4010E3B1223
:1081E000D8B443D0020E18EC02F0E86A44B2010F92
:1081F00083BC010819E0448283AC449245A002D0BC
:108200004A4A4B2A45A204D0010E4A5E000E4B5A40
:10821000E86A81B6010F81B8010804E193968A9655
:1082200093988A980301516B0001E86A44B4010FE6
:1082300083BE010819E0448483AE449445A402D06F
:108240004C4A4D2A45A604D0010E4C5E000E4D5AF4
:10825000E86A81BC010F81BA010804E1939A8A9A05
:10826000939C8A9C0301526B00011200840E026EE3
:10827000020E086E840E036E010E046E050E096E6A
:10828000D451136EEFEC01F0D551136EEFEC01F009
:10829000D651136EEFEC01F0D751136EEFEC01F0F5
:1082A000D851136EEFEC01F0D951136EEFEC01F0E1
:1082B00096948D8496948D941200000100C031F440
:1082C00001C032F4A9CF33F4AACF34F4A6CF35F4E9
:1082D000A7CF36F4A8CF37F4EACF38F4E9CF39F492
:1082E000E2CF3AF4E1CF3BF413C03CF414C03DF4C8
:1082F0001FC03EF420C03FF421C040F4F3CF41F44E
:108300003BC042F49EAA54D0AECFA9F0610EA95D45
:10831000000ED8B0010E3B6E7B0EA95D02E3000E8D
:1083200001D0010E3B1601E0A99B9A3103E3A9514C
:10833000BBEC01F09E9A0A0EA95D17E001EE47F032
:10834000EE50FEE1ED52A9C0EEFFEF6A4E0E0301C2
:10835000505D000104E20301502B000105D0030130
:10836000506B01EE47F0EF6A0001240EA95D08E1B1
:1083700001EE47F0EF6A01EE47F0A9C0EEFFEF6AA9
:108380000D0EA95D15E1448C0301506B0001D20E66
:10839000AB6F00EEF6F011EE47F0500EE75204E03E
:1083A000E6CFEEFFE82EFAD7EF6A01EE47F0EF6A6C
:1083B000F0A22AD00EEC00F093968A9693988A98B1
:1083C000939A8A9A939C8A9C95968C96AA6AA96A93
:1083D0004A50D3EC01F04B50D3EC01F0AA6A020EE4
:1083E000A96E4C50D3EC01F04D50D3EC01F0AA6AC9
:1083F000210EA96E03018951D3EC01F003018A51CA
:10840000D3EC01F00001FED731C400F032C401F01A
:1084100033C4A9FF34C4AAFF35C4A6FF36C4A7FFDE
:1084200037C4A8FF38C4EAFF39C4E9FF3AC4E2FF01
:108430003BC4E1FF3CC413F03DC414F03EC41FF044
:108440003FC420F040C421F041C4F3FF42C43BF0DC
:108450001100F29EE0CF43F43BC044F4D8CF45F482
:10846000E8CF46F4F28E00019EA468D09E949F2B24
:108470000F0E9F5DD8A062D09F6B000E45B8010E15
:10848000010AD8B44598D8A44588000E43B0010E1F
:108490003B6E000E42BE010E3B120DE0AA2B0D0EEC
:1084A000AA5D09E34390429E0301516B526B0001A8
:1084B000AA6B42904292FA0E03015B5D000102E258
:1084C00003015B2B03015453000102E00301540735
:1084D000000144BE2BD0000E81B6010E3B6E000E93
:1084E00081B8010E3B1202E00301512B0001000E86
:1084F00081BA010E3B6E000E81BC010E3B1202E000
:108500000301522B050E0301515D000105E3428E6C
:1085100093988A9893968A96050E0301525D0001FE
:1085200005E34380939A8A9A939C8A9CBE0E03012A
:10853000875D000102E20301872B0001F29E43C424
:10854000E0FF44C43BF045C4D8FF46C4E8FFF28EC8
:108550001000AA6A040EA96EE8EC01F0676FE8EC5F
:1085600001F0686FAA6A060EA96EE8EC01F0696F67
:10857000E8EC01F06A6FAA6A080EA96EE8EC01F057
:108580006F6FE8EC01F0706FAA6A0A0EA96EE8EC52
:1085900001F0716FE8EC01F0726FAA6A0C0EA96E1F
:1085A000E8EC01F0736FE8EC01F0746FAA6A0E0E4C
:1085B000A96EE8EC01F0666FAA6A0F0EA96EE8ECEE
:1085C00001F09A6FAA6A100EA96EE8EC01F003019F
:1085D000596FAA6A110EA96EE8EC01F00301556FFC
:1085E000AA6A120EA96EE8EC01F003013A6FE8ECFA
:1085F00001F003013B6FE8EC01F003013C6FE8EC94
:1086000001F003013D6FAA6A160EA96EE8EC01F0B5
:1086100003013E6FE8EC01F003013F6FE8EC01F06D
:108620000301406FE8EC01F00301416FAA6A1A0EE2
:10863000A96EE8EC01F00301426FE8EC01F00301E0
:10864000436FAA6A1C0EA96EE8EC01F00301856F66
:10865000E8EC01F00301866FC30E146E500E136E2A
:1086600086C318F085C317F068EC02F00301836F2E
:1086700014C084F386510A0DF3CF86F385510A0D99
:10868000F3CF85F3F4508627020E555DD8A4010E72
:108690003B6E040E555DD8A4010E3B160A0E555DC7
:1086A000D8A4010E3B16140E555DD8A4010E3B163E
:1086B000000103E00301040E556F00014BC057F0A9
:1086C0004AC056F04DC059F04CC058F00301555106
:1086D000B40DF3CFC4F0F4CFC5F05551680DF3CF0E
:1086E000C6F0F4CFC7F00001C72766510301550358
:1086F000F4CFC9F0F3CFC8F055510A0DF3CFCAF04B
:10870000F4CFCBF05551640DF3CFCCF0F4CFCDF0D6
:1087100055511E0DF3CFD0F0F4CFD1F05551320D9D
:10872000F3CFCEF0F4CFCFF055510F0DF3CFD2F001
:10873000F4CFD3F000011200800E016EC00E19ECD0
:1087400000F0200E43EC01F0000E43EC01F0200E8F
:1087500043EC01F04D0E43EC01F0200E43EC01F030
:10876000010E43EC01F0200E43EC01F043EC01F06C
:1087700043EC01F0040E43EC01F0200E43EC01F059
:1087800043EC01F043EC01F043EC01F0000E43EC4C
:1087900001F0200E43EC01F0560E43EC01F0200EE8
:1087A00043EC01F0010E43EC01F0200E43EF01F029
:1087B000800E016EC00E19EC00F0200E43EC01F0AB
:1087C000000E43EC01F0200E43EC01F04D0E43ECA3
:1087D00001F0200E43EC01F0010E43EC01F0200EFD
:1087E00043EC01F043EC01F043EC01F0040E43ECE8
:1087F00001F01F0EF76EDC0EF66E3BEF01F0080E77
:10880000B86EAC98AC8403018851880DF3CF6DF33A
:10881000F4CF6EF36F6B706B8851130DF3506E27AE
:10882000F4506F23000E7023B9C014F0B8C013F0D9
:10883000186A640E176E68EC02F00001906F14C0A5
:1088400091F070C329F06FC328F06EC327F06DC399
:1088500026F029C016F028C015F027C014F026C055
:1088600013F090C01BF091C01CF01D6A1E6A3DEC15
:1088700002F016C029F015C028F014C027F013C06C
:1088800026F02606000E275A285A295A2830273063
:10889000916F2630906F91C0B0FF90C0AFFF120073
:1088A000FFD7FFD7B76BB66BB7530CE1640EB65D5D
:1088B00009E2030E18EC02F0CBEC40F0B62B000EF0
:1088C000B723F2E31200030155518F03F3CF46F0B3
:1088D000F4CF47F09003F350472642804850000100
:1088E000C85D4950C9594950C919D8B0800A19E61C
:1088F0004850C45D486E4950C559496EC45146261A
:10890000C5514722C651465CC75147584750C71901
:10891000D8B0800A06E7C651465C466EC751475834
:10892000476E47C09AF346C099F333D89CC35FF0B3
:108930009BC35EF047C092F346C091F3120003015F
:1089400055519303F3CF97F3F4CF98F39403F35077
:108950009827428297510001C85D03019851000198
:10896000C959030198510001C919D8B0800A0BE612
:10897000030197510001C45D0301976F98510001F5
:10898000C5590301986F000198C396F397C395F3F7
:1089900012009A51E8A616D0C4510301995D9D6F4B
:1089A0000001C55103019A599E6F9E510001E8AE26
:1089B00007D0C65103019D270001C75103019E2323
:1089C000000104D09AC39EF399C39DF36F51030134
:1089D0009D270001705103019E2300019A35D8A004
:1089E000C3D07451E8BE11D0120E745D0EE303E1E2
:1089F0005D0E735D0AE3AA6A0C0EA96EE8EC01F045
:108A00000001736FE8EC01F0746FC65103019D25FE
:108A10000B6E0001C75103019E210C6E00017351C2
:108A20000B5C74510C580C507419D8B0800A02E7D2
:108A3000000E01D0010E3B6E030155510E0DF3CF18
:108A400026F0F4CF27F0286A2726000E282255AFFB
:108A500004D00E0E275E010E285A0001296A28BE96
:108A600029066F5126240B6E705127200C6E000EC4
:108A700070BFFF0E28200D6E000E70BFFF0E292064
:108A80000E6E4AC013F04BC014F0000E14BEFF0E61
:108A9000156E166E13500B5C14500C5815500D5873
:108AA00016500E5816500E18D8B0800A02E7000E65
:108AB00001D0010E3B1607E0C65103019D270001BE
:108AC000C75103019E2300016F51CE250B6E7051DB
:108AD000CF210C6E000E0CBEFF0E0D6E0E6E4AC046
:108AE00013F04BC014F0000E14BEFF0E156E166E80
:108AF0000B50135C0C5014580D5015580E5016584E
:108B00000E501618D8B0800A02E7000E01D0010EF0
:108B10003B6EC65103019D5D0B6E0001C751030101
:108B20009E590C6E000E55BFFF0E0C5C07E00C50FA
:108B30005519D8B0800A800B07E008D000010B500F
:108B40000301555D000102E3000E01D0010E3B164A
:108B5000000109E0C65103019D5D9D6F0001C751F1
:108B600003019E599E6F00019EC39CF39DC39BF31E
:108B70001200A66B03019F53000118E000EEF6F00F
:108B8000A651EB500B6E2C0E0B5CD8A4010E3B6E65
:108B9000500EA65D010ED8B0000E3B1602E0A62BCB
:108BA000EDD7A62B03019F070001E4D7A56B00EECC
:108BB000F6F0A651EB500B6E2C0E0B5C10E000EEA5
:108BC000F6F0A651EBCF0BF003EEC4F0A5510BC0AD
:108BD000EBFF4E0EA55D01E2A52BA62BE8D7F36AAD
:108BE00003EEC4F0A551F3CFEBFF12000301A05137
:108BF00016EC09F0396A386A340E376E850E366E17
:108C00006FEC08F035C0ACF334C0ABF333C0AAF35B
:108C100032C0A9F30301A0510E085A6F0001010EE2
:108C200082B6000E3B6E010E82B4000E3B12010EA6
:108C300080BC000E3B12010E80BE000E3B1201E014
:108C4000EDD782A205EF4BF05AC3BEF3A0C3BFF32A
:108C5000A4C3C3F3A3C3C2F3A2C3C1F3A1C3C0F3AC
:108C6000F3EC4BF080BCB9D10C0E03015A5D010E40
:108C7000D8A4000E3B6E020EA05D010ED8A4000E1B
:108C80003B16A4C335F0A3C334F0A2C333F0A1C391
:108C900032F0396A386A480E376E850E366EBFEC90
:108CA00006F03B16000118E0396A386A480E376E44
:108CB000850E366EA4C335F0A3C334F0A2C333F0DF
:108CC000A1C332F079EC07F035C0A4F334C0A3F3AC
:108CD00033C0A2F332C0A1F30D0E03015A5D010EA1
:108CE000D8A4000E3B6EA4C335F0A3C334F0A2C3D6
:108CF00033F0A1C332F0396A386A200E376E820E23
:108D0000366EBFEC06F03B16000118E0396A386A8F
:108D1000200E376E820E366EA4C335F0A3C334F036
:108D2000A2C333F0A1C332F079EC07F035C0A4F34D
:108D300034C0A3F333C0A2F332C0A1F30E0E03017B
:108D40005A5D010ED8A4000E3B6EA4C335F0A3C338
:108D500034F0A2C333F0A1C332F0396A386A376AFB
:108D60007F0E366EBFEC06F03B16000117E0396A45
:108D7000386A376A7F0E366EA4C335F0A3C334F069
:108D8000A2C333F0A1C332F079EC07F035C0A4F3ED
:108D900034C0A3F333C0A2F332C0A1F3100E030119
:108DA0005A5D010ED8A4000E3B6EA4C335F0A3C3D8
:108DB00034F0A2C333F0A1C332F0CD0E396ECC0E25
:108DC000386E4C0E376E7B0E366EBFEC06F03B16DF
:108DD00000011AE0CD0E396ECC0E386E4C0E376E97
:108DE0007B0E366EA4C335F0A3C334F0A2C333F0B8
:108DF000A1C332F079EC07F035C0A4F334C0A3F37B
:108E000033C0A2F332C0A1F3110E03015A5D010E6B
:108E1000D8A4000E3B6EA4C335F0A3C334F0A2C3A4
:108E200033F0A1C332F00A0E396ED70E386E230E1E
:108E3000376E780E366EBFEC06F03B1600011AE076
:108E40000A0E396ED70E386E230E376E780E366ED8
:108E5000A4C335F0A3C334F0A2C333F0A1C332F0EE
:108E600079EC07F035C0A4F334C0A3F333C0A2F308
:108E700032C0A1F3120E03015A5D010ED8A4000EF8
:108E80003B6EA4C335F0A3C334F0A2C333F0A1C337
:108E900032F06F0E396E120E386E030E376E750E8D
:108EA000366EBFEC06F03B1600011AE06F0E396E0D
:108EB000120E386E030E376E750E366EA4C335F083
:108EC000A3C334F0A2C333F0A1C332F079EC07F0AE
:108ED00035C0A4F334C0A3F333C0A2F332C0A1F36E
:108EE000130E03015A5D010ED8A4000E3B6EA4C3FD
:108EF00035F0A3C334F0A2C333F0A1C332F0170E90
:108F0000396EB70E386E510E376E710E366EBFEC7D
:108F100006F03B1600011AE0170E396EB70E386ED8
:108F2000510E376E710E366EA4C335F0A3C334F004
:108F3000A2C333F0A1C332F079EC07F035C0A4F33B
:108F400034C0A3F333C0A2F332C0A1F3140E030163
:108F50005A5D010ED8A4000E3B6EA4C335F0A3C326
:108F600034F0A2C333F0A1C332F0AC0E396EC50E9B
:108F7000386E270E376E6E0E366EBFEC06F03B165F
:108F800000011AE0AC0E396EC50E386E270E376E32
:108F90006E0E366EA4C335F0A3C334F0A2C333F013
:108FA000A1C332F079EC07F035C0A4F334C0A3F3C9
:108FB00033C0A2F332C0A1F345985AC3BEF3A0C395
:108FC000BFF3A4C3C3F3A3C3C2F3A2C3C1F3A1C33A
:108FD000C0F3F3EC4BF080ACFED780BEB3EF4AF0A9
:108FE0000C0E03015A5D010ED8A4000E3B6E020E5A
:108FF000A05D010ED8A4000E3B160001D8B44DD0E0
:10900000396A386A480E376E850E366EACC335F055
:10901000ABC334F0AAC333F0A9C332F079EC07F044
:1090200035C00EF034C00DF033C00CF032C00BF080
:10903000A4C335F0A3C334F0A2C333F0A1C332F00C
:109040000EC039F00DC038F00CC037F00BC036F050
:10905000F7EC06F0010819E0356A346A480E336E01
:10906000850E326EA4C339F0A3C338F0A2C337F023
:10907000A1C336F07BEC07F035C0A4F334C0A3F3F2
:1090800033C0A2F332C0A1F308D0ACC3A4F3ABC386
:10909000A3F3AAC3A2F3A9C3A1F30D0E03015A5D62
:1090A0000001D8A44DD0396A386A200E376E820E7E
:1090B000366EACC335F0ABC334F0AAC333F0A9C3EA
:1090C00032F079EC07F035C00EF034C00DF033C04B
:1090D0000CF032C00BF0A4C335F0A3C334F0A2C32C
:1090E00033F0A1C332F00EC039F00DC038F00CC01F
:1090F00037F00BC036F0F7EC06F0010819E0356ADE
:10910000346A200E336E820E326EA4C339F0A3C3CC
:1091100038F0A2C337F0A1C336F07BEC07F035C0BE
:10912000A4F334C0A3F333C0A2F332C0A1F308D038
:10913000ACC3A4F3ABC3A3F3AAC3A2F3A9C3A1F323
:109140000E0E03015A5D0001D8A44BD0396A386A6B
:10915000376A7F0E366EACC335F0ABC334F0AAC3AA
:1091600033F0A9C332F079EC07F035C00EF034C00B
:109170000DF033C00CF032C00BF0A4C335F0A3C324
:1091800034F0A2C333F0A1C332F00EC039F00DC0E9
:1091900038F00CC037F00BC036F0F7EC06F00108E1
:1091A00018E0356A346A336A7F0E326EA4C339F030
:1091B000A3C338F0A2C337F0A1C336F07BEC07F0AD
:1091C00035C0A4F334C0A3F333C0A2F332C0A1F37B
:1091D00008D0ACC3A4F3ABC3A3F3AAC3A2F3A9C33F
:1091E000A1F3100E03015A5D0001D8A451D0CD0E99
:1091F000396ECC0E386E4C0E376E7B0E366EACC3AD
:1092000035F0ABC334F0AAC333F0A9C332F079EC24
:1092100007F035C00EF034C00DF033C00CF032C092
:109220000BF0A4C335F0A3C334F0A2C333F0A1C341
:1092300032F00EC039F00DC038F00CC037F00BC062
:1092400036F0F7EC06F001081BE0CD0E356ECC0EC3
:10925000346E4C0E336E7B0E326EA4C339F0A3C352
:1092600038F0A2C337F0A1C336F07BEC07F035C06D
:10927000A4F334C0A3F333C0A2F332C0A1F308D0E7
:10928000ACC3A4F3ABC3A3F3AAC3A2F3A9C3A1F3D2
:10929000110E03015A5D0001D8A451D00A0E396E97
:1092A000D70E386E230E376E780E366EACC335F09F
:1092B000ABC334F0AAC333F0A9C332F079EC07F0A2
:1092C00035C00EF034C00DF033C00CF032C00BF0DE
:1092D000A4C335F0A3C334F0A2C333F0A1C332F06A
:1092E0000EC039F00DC038F00CC037F00BC036F0AE
:1092F000F7EC06F001081BE00A0E356ED70E346E4F
:10930000230E336E780E326EA4C339F0A3C338F047
:10931000A2C337F0A1C336F07BEC07F035C0A4F34D
:1093200034C0A3F333C0A2F332C0A1F308D0ACC35E
:10933000A4F3ABC3A3F3AAC3A2F3A9C3A1F3120E70
:1093400003015A5D0001D8A451D06F0E396E120E80
:10935000386E030E376E750E366EACC335F0ABC388
:1093600034F0AAC333F0A9C332F079EC07F035C06A
:109370000EF034C00DF033C00CF032C00BF0A4C3BB
:1093800035F0A3C334F0A2C333F0A1C332F00EC052
:1093900039F00DC038F00CC037F00BC036F0F7ECE8
:1093A00006F001081BE06F0E356E120E346E030ED0
:1093B000336E750E326EA4C339F0A3C338F0A2C366
:1093C00037F0A1C336F07BEC07F035C0A4F334C00E
:1093D000A3F333C0A2F332C0A1F308D0ACC3A4F30B
:1093E000ABC3A3F3AAC3A2F3A9C3A1F3130E030152
:1093F0005A5D0001D8A451D0170E396EB70E386EE1
:10940000510E376E710E366EACC335F0ABC334F00F
:10941000AAC333F0A9C332F079EC07F035C00EF0DF
:1094200034C00DF033C00CF032C00BF0A4C335F0E3
:10943000A3C334F0A2C333F0A1C332F00EC039F09D
:109440000DC038F00CC037F00BC036F0F7EC06F06A
:1094500001081BE0170E356EB70E346E510E336ED9
:10946000710E326EA4C339F0A3C338F0A2C337F033
:10947000A1C336F07BEC07F035C0A4F334C0A3F3EE
:1094800033C0A2F332C0A1F308D0ACC3A4F3ABC382
:10949000A3F3AAC3A2F3A9C3A1F3140E03015A5D57
:1094A0000001D8A451D0AC0E396EC50E386E270E0F
:1094B000376E6E0E366EACC335F0ABC334F0AAC354
:1094C00033F0A9C332F079EC07F035C00EF034C0A8
:1094D0000DF033C00CF032C00BF0A4C335F0A3C3C1
:1094E00034F0A2C333F0A1C332F00EC039F00DC086
:1094F00038F00CC037F00BC036F0F7EC06F001087E
:109500001BE0AC0E356EC50E346E270E336E6E0E3C
:10951000326EA4C339F0A3C338F0A2C337F0A1C39D
:1095200036F07BEC07F035C0A4F334C0A3F333C0AE
:10953000A2F332C0A1F308D0ACC3A4F3ABC3A3F32E
:10954000AAC3A2F3A9C3A1F35AC3BEF3A0C3BFF336
:10955000A4C3C3F3A3C3C2F3A2C3C1F3A1C3C0F3A3
:1095600042D980AEFED782B62AD003015A07A05155
:109570000D080B6E000ED8A0FF0F0C6E0C5204E10C
:109580005A510B5C000103E30301140E5A6F0F0ED6
:1095900003015A5D000102E103015A0700014588F9
:1095A0005AC3BEF3A0C3BFF3A4C3C3F3A3C3C2F3A0
:1095B000A2C3C1F3A1C3C0F316D982A6FED782B459
:1095C00022D003015A2B150E5A5D000104E303015A
:1095D000A0510E085A6F0F0E03015A5D000102E1FF
:1095E00003015A2B000145885AC3BEF3A0C3BFF341
:1095F000A4C3C3F3A3C3C2F3A2C3C1F3A1C3C0F303
:10960000F2D882A4FED721EF46F0A4C3A8F3A3C3E7
:10961000A7F3A2C3A6F3A1C3A5F382A2FED71200AB
:109620000301AF6B030E0301AF5D000113E204EE13
:1096300015F00301AF51EB50BD6F0001C0D845BE1E
:1096400005D00301AE69AD69000112000301AF2B23
:109650000001E8E301EE98F020EC00F00301AD6FAB
:109660001CC0AEF3000112000301BC6BBB6BBA6BF4
:10967000B96BB76BB66BB56BB46BB86B000104EE2E
:109680001CF00301B851EB500B6E0B520001D8B423
:1096900079D004EE1CF00301B851EB50BD6F00010E
:1096A0008ED845AE5AD0BCC329F0BBC328F0BAC38C
:1096B00027F0B9C326F029C016F028C015F027C03E
:1096C00014F026C013F01E6A1D6A1C6A0A0E1B6E77
:1096D000BAEC02F016C029F015C028F014C027F02B
:1096E00013C026F004EE1CF00301B851EB500B6ED2
:1096F0002D6A2C6A2B6A0BC02AF00F0E2A142A6ED0
:10970000000E2B142B6E000E2C142C6E000E2D143C
:109710002D6E2A502624B96F2B502720BA6F2C505B
:109720002820BB6F2D502920BC6F356A346A200E6B
:10973000336E820E326EB7C339F0B6C338F0B5C39C
:1097400037F0B4C336F06FEC08F035C0B7F334C06F
:10975000B6F333C0B5F332C0B4F3000104EE1CF02D
:109760000301B851EB500B6E2E0E0B5C000106E1AD
:109770000301B76BB66BB56B7F0EB46F0301B82BEB
:1097800000017CD7B7C339F0B6C338F0B5C337F0A2
:10979000B4C336F0BCC335F0BBC334F0BAC333F046
:1097A000B9C332F01AEC09F009EC08F035C0B3F394
:1097B00034C0B2F333C0B1F332C0B0F31200300E94
:1097C0000301BD5D000ED8B0010E3B6E3A0EBD5DCB
:1097D000000102E3000E01D0010E3B1602E0458EAF
:1097E00001D0459E1200010E0301BF5D00010AE198
:1097F00001EEFCF01F0EF76EE80EF66E26EC03F09D
:10980000EF6A23D001EEFCF01F0EF76EF60EF66E37
:1098100026EC03F0EF6AC3C335F0C2C334F0C1C312
:1098200033F0C0C332F0396A386A480E376E850E9D
:10983000366EBFEC06F0010808E001EEFCF0EE50D9
:10984000FEE1ED52300EEE6EEF6AC3C335F0C2C3D7
:1098500034F0C1C333F0C0C332F0396A386A200E25
:10986000376E820E366EBFEC06F0010808E001EE9E
:10987000FCF0EE50FEE1ED52300EEE6EEF6A01EEBE
:10988000FCF0EE50FEE1ED52020E016EC3C329F072
:10989000C2C328F0C1C327F0C0C326F0050EA7EC51
:1098A00000F0EF6A45A809D00301BE05FC0FE96E80
:1098B000010EEA6AEA22200EEF6E0001800E016EB0
:1098C00019EC00F001EEFCF0EE5003E043EC01F087
:1098D000FBD7800E016EC00E19EC00F0200E43EC99
:1098E00001F0030E43EC01F0200E43EC01F0500EAA
:1098F00043EC01F0200E43EC01F0020E43EC01F0CA
:10990000200EF76E020EF66E3BEC01F0000E43ECFB
:1099100001F0200E43EC01F0560E43EC01F0200E56
:1099200043EC01F0010E43EC01F0200E43EF01F097
:020000040030CA
:03000100D80F38DD
:020005003D803C
:0600080008C00FE00F40EC
:0200000400F00A
:100000006C001800F80200006C00180068065AF82E
:10001000460484410F7E831E8FC5CC00FA00FF800A
:0400200025000000B7
:00000001FF
